:020000040000FA
:0408000046EF0CF0C3
:1008100003B275EF05F0F2B493EF05F09EB09BEFD5
:1008200005F09EB2A3EF05F0F2A81AEF04F0F2B2C1
:1008300023EF04F0F2B01FEF04F0F5EF0BF0F296A7
:10084000F290F5EF0BF0CD90F2929EA02DEF04F018
:100850000101533F2DEF04F0542BB2C1B6F1B3C1E7
:10086000B7F1B4C1B8F1B5C1B9F1AEC1B2F1AFC120
:10087000B3F1B0C1B4F1B1C1B5F1AAC1AEF1ABC130
:10088000AFF1ACC1B0F1ADC1B1F1A6C1AAF1A7C140
:10089000ABF1A8C1ACF1A9C1ADF1A2C1A6F1A3C150
:1008A000A7F1A4C1A8F1A5C1A9F19EC1A2F19FC160
:1008B000A3F1A0C1A4F1A1C1A5F19AC19EF19BC170
:1008C0009FF19CC1A0F19DC1A1F1CECF9AF1CFCFF4
:1008D0009BF153C19CF154C19DF1CF6ACE6A0101D5
:1008E000536B546B9E90CD800FBC0F8E0FBA7CEF74
:1008F00004F00F8AF5EF0BF013880F8C0FBEB9EFE1
:1009000004F09AC19EF19BC19FF19CC1A0F19DC1D1
:10091000A1F19EC1A2F19FC1A3F1A0C1A4F1A1C107
:10092000A5F1A2C1A6F1A3C1A7F1A4C1A8F1A5C1D7
:10093000A9F1A6C1AAF1A7C1ABF1A8C1ACF1A9C1A7
:10094000ADF1AAC1AEF1ABC1AFF1ACC1B0F1ADC177
:10095000B1F1AEC1B2F1AFC1B3F1B0C1B4F1B1C147
:10096000B5F1B2C1B6F1B3C1B7F1B4C1B8F1B5C117
:10097000B9F101015E6B5F6B606B616B9A515E2731
:100980009B515F239C5160239D5161239E515E27A3
:100990009F515F23A0516023A1516123A2515E2783
:1009A000A3515F23A4516023A5516123A6515E2763
:1009B000A7515F23A8516023A9516123AA515E2743
:1009C000AB515F23AC516023AD516123AE515E2723
:1009D000AF515F23B0516023B1516123B2515E2703
:1009E000B3515F23B4516023B5516123B6515E27E3
:1009F000B7515F23B8516023B9516123D8900101E9
:100A0000613360335F335E33D8900101613360330B
:100A10005F335E33D8900101613360335F335E33FF
:100A200000C10CF101C10DF102C10EF103C10FF1C2
:100A300004C110F105C111F106C112F107C113F192
:100A400008C114F109C115F10AC116F10BC117F162
:100A500034C135F111B838EF05F00101620E046FB1
:100A6000010E056F000E066F000E076F41EF05F0D7
:100A70000101A70E046F020E056F000E066F000E37
:100A8000076F5EC100F15FC101F160C102F161C198
:100A900003F182EC3BF003BF04D01DBE02D01DA0C9
:100AA000108C11A059EF05F010BA59EF05F00F8026
:100AB000108A0CC100F10DC101F10EC102F10FC18C
:100AC00003F110C104F111C105F112C106F113C106
:100AD00007F114C108F115C109F116C10AF117C1D6
:100AE0000BF135C134F1F5EF0BF00392ABB2AB98DB
:100AF000AB88030103EE00F080517F0BE92604C0B0
:100B0000EFFF802B8151805D700BD8A48B82000099
:100B10008051815D700BD8A48B9281518019D8B41B
:100B20000790F5EF0BF0F2940101453FF5EF0BF064
:100B3000462BF5EF0BF09E900101533FF5EF0BF0C4
:100B4000542BF5EF0BF09E9211B89AEF08F00400C9
:100B500066A1ABEF05F08BB4B5EF05F010ACB5EFC7
:100B600005F08B84109CB6EF05F08B9407B40DEF65
:100B700006F007B00DEF06F01EC620F61FC621F6E0
:100B80001CC61EF61DC61FF61AC61CF61BC61DF691
:100B900006C608F607C609F604C606F605C607F631
:100BA00002C604F603C605F626C628F627C629F6A9
:100BB00024C626F625C627F622C624F623C625F621
:100BC0000EC610F60FC611F60CC60EF60DC60FF6C1
:100BD0000AC60CF60BC60DF62EC630F62FC631F639
:100BE0002CC62EF62DC62FF62AC62CF62BC62DF6B1
:100BF00016C618F617C619F614C616F615C617F651
:100C000012C614F613C615F616B0E8EC3DF01EEC4D
:100C10003DF096EC3DF044EC3DF0077C07AC28EF4E
:100C200006F0C274C2B422EF06F0C3CFB7F5C4CF4A
:100C3000B8F50501D890B833B733D890B833B73387
:100C400029EF06F0C3CF55F1C4CF56F129EF06F0D6
:100C5000C28207B49BEF06F047C14BF148C14CF18B
:100C600049C14DF14AC14EF15EC162F15FC163F10C
:100C700060C164F161C165F113A841EF06F0138C06
:100C800013989AC1BAF19BC1BBF19CC1BCF19DC143
:100C9000BDF19EC1BEF19FC1BFF1A0C1C0F1A1C114
:100CA000C1F1A2C1C2F1A3C1C3F1A4C1C4F1A5C1E4
:100CB000C5F1A6C1C6F1A7C1C7F1A8C1C8F1A9C1B4
:100CC000C9F1AAC1CAF1ABC1CBF1ACC1CCF1ADC184
:100CD000CDF1AEC1CEF1AFC1CFF1B0C1D0F1B1C154
:100CE000D1F1B2C1D2F1B3C1D3F1B4C1D4F1B5C124
:100CF000D5F1B6C1D6F1B7C1D7F1B8C1D8F1B9C1F4
:100D0000D9F1B7C5B9F5B8C5BAF5B9C5BBF5BAC516
:100D1000BCF5010155515B2756515C23E86A5D2300
:100D20000E2E9BEF06F05CC157F15DC158F15B6B75
:100D30005C6B5D6B078E0201002FF5EF0BF03C0E34
:100D4000006F1E50E00BE00AE86612881CBE02D05D
:100D50001CB4108E00C10CF101C10DF102C10EF1E5
:100D600003C10FF104C110F105C111F106C112F167
:100D700007C113F108C114F109C115F10AC116F137
:100D80000BC117F134C135F181AA03EF07F015A4A7
:100D90004EEF07F005012F51000AD8B491EF07F08C
:100DA00005012F51010AD8B40DEF07F005012F51AD
:100DB000020AD8B44EEF07F005012F51030AD8B448
:100DC0004EEF07F005012F51040AD8B44EEF07F09B
:100DD00005012F51050AD8B44EEF07F005012F5138
:100DE000060AD8B44EEF07F005012F51070AD8B410
:100DF0004EEF07F005012F51320AD8B40BEF07F080
:100E00002F6B91EF07F000011750030AD8B44EEF93
:100E100007F091EF07F091EF07F00501576718EF22
:100E200007F0586718EF07F0596718EF07F05A678F
:100E30001CEF07F091EF07F05BC500F15CC501F115
:100E40005DC502F15EC503F10101010E046F000EE4
:100E5000056F000E066F000E076F82EC3BF000C1BD
:100E60005BF501C15CF502C15DF503C15EF50101F1
:100E7000006742EF07F0016742EF07F0026742EFB9
:100E800007F0036791EF07F057C55BF558C55CF5B0
:100E900059C55DF55AC55EF57BEF07F00FBE63EFF0
:100EA00007F010A068EF07F0010147675FEF07F058
:100EB00048675FEF07F049675FEF07F04A6763EF46
:100EC00007F068EF07F007AE68EF07F07BEF07F079
:100ED0000501312F91EF07F03C0E316F302F91EF6C
:100EE00007F00101000E626FE00E636FA50E646FE4
:100EF000010E656F138800011750000AD8B489EFFE
:100F000007F000011750030AD8B48EEF07F091EFF5
:100F100007F00001010E176E91EF07F00001040EBB
:100F2000176E0501666B37B797EF07F066810CC146
:100F300000F10DC101F10EC102F10FC103F110C1A9
:100F400004F111C105F112C106F113C107F114C179
:100F500008F115C109F116C10AF117C10BF135C12C
:100F600034F100C10CF101C10DF102C10EF103C158
:100F70000FF104C110F105C111F106C112F107C151
:100F800013F108C114F109C115F10AC116F10BC121
:100F900017F134C135F101018E67D6EF07F08F6785
:100FA000D6EF07F09067D6EF07F09167DAEF07F01A
:100FB0000BEF08F092C100F193C101F194C102F16D
:100FC00095C103F10101010E046F000E056F000EC3
:100FD000066F000E076F82EC3BF000C192F101C179
:100FE00093F102C194F103C195F10101006700EF93
:100FF00008F0016700EF08F0026700EF08F00367F0
:101000000BEF08F08EC192F18FC193F190C194F172
:1010100091C195F10F80D57ED5BE6ED0D6CF47F168
:10102000D7CF48F145C149F1E86AE8CF4AF1138AC0
:101030001DBE02D01DA0108C109047C100F148C108
:1010400001F149C102F14AC103F101010A0E046F25
:10105000000E056F000E066F000E076F82EC3BF06E
:1010600003AF1080010154A742EF08F00F9A0F9CC4
:101070000F9E0101000E5E6F600E5F6F3D0E606F90
:10108000080E616F010147BF52EF08F0486752EF49
:1010900008F0496752EF08F04A6752EF08F0F2880B
:1010A00077EF08F0F2985E6B5F6B606B616B9A6B29
:1010B0009B6B9C6B9D6B9E6B9F6BA06BA16BA26BE4
:1010C000A36BA46BA56BA66BA76BA86BA96BAA6B94
:1010D000AB6BAC6BAD6BAE6BAF6BB06BB16BB26B44
:1010E000B36BB46BB56BB66BB76BB86BB96BD76AD8
:1010F000D66A0101456B466B0CC100F10DC101F1CF
:101100000EC102F10FC103F110C104F111C105F1CB
:1011100012C106F113C107F114C108F115C109F19B
:1011200016C10AF117C10BF135C134F1F5EF0BF01F
:10113000F5EF0BF00201002F02EF0BF0D59ED6CF9A
:1011400047F1D7CF48F145C149F1E86AE8CF4AF104
:10115000138AD76AD66A0101456B466BD58E1E503D
:10116000E00BE00AE86612881CBE02D01CB4108EA8
:101170001BAE208C00C10CF101C10DF102C10EF1BA
:1011800003C10FF104C110F105C111F106C112F143
:1011900007C113F108C114F109C115F10AC116F113
:1011A0000BC117F134C135F10FA0109A11B8E4EF5B
:1011B00008F00101620E046F010E056F000E066F4C
:1011C000000E076FEDEF08F00101A70E046F020E8D
:1011D000056F000E066F000E076F47C100F148C192
:1011E00001F149C102F14AC103F182EC3BF003BFB6
:1011F00000EF09F01DBE02D01DA0108C11B00F80B1
:101200000CC100F10DC101F10EC102F10FC103F1DA
:1012100010C104F111C105F112C106F113C107F1AA
:1012200014C108F115C109F116C10AF117C10BF17A
:1012300035C134F102013C0E006F00C10CF101C157
:101240000DF102C10EF103C10FF104C110F105C18E
:1012500011F106C112F107C113F108C114F109C15E
:1012600015F10AC116F10BC117F134C135F181BA7C
:101270003DEF09F015B27CEF09F015A07CEF09F005
:1012800015A4C7EF09F005012F51000AD8B40AEFE1
:101290000AF005012F51010AD8B486EF09F00501C3
:1012A0002F51020AD8B4C7EF09F005012F51030AE4
:1012B000D8B4C7EF09F005012F51040AD8B4C7EF1D
:1012C00009F005012F51050AD8B4C7EF09F005014F
:1012D0002F51060AD8B4C7EF09F005012F51070AAC
:1012E000D8B4C7EF09F005012F51320AD8B484EF02
:1012F00009F02F6B0AEF0AF000011750030AD8B467
:10130000C7EF09F00AEF0AF00AEF0AF00501576784
:1013100091EF09F0586791EF09F0596791EF09F0E3
:101320005A6795EF09F00AEF0AF05BC500F15CC55A
:1013300001F15DC502F15EC503F10101010E046F0B
:10134000000E056F000E066F000E076F82EC3BF07B
:1013500000C15BF501C15CF502C15DF503C15EF53D
:1013600001010067BBEF09F00167BBEF09F00267FD
:10137000BBEF09F003670AEF0AF057C55BF558C5E4
:101380005CF559C55DF55AC55EF5F4EF09F00FBE81
:10139000DCEF09F010A0E1EF09F001014767D8EF99
:1013A00009F04867D8EF09F04967D8EF09F04A67B4
:1013B000DCEF09F0E1EF09F007AEE1EF09F0F4EF3F
:1013C00009F00501312F0AEF0AF03C0E316F302F82
:1013D0000AEF0AF00101000E626FE00E636FA50EC6
:1013E000646F010E656F138800011750000AD8B4AE
:1013F00002EF0AF000011750030AD8B407EF0AF011
:101400000AEF0AF00001010E176E0AEF0AF0000160
:10141000040E176E0501666B37B710EF0AF0668190
:101420000CC100F10DC101F10EC102F10FC103F1B8
:1014300010C104F111C105F112C106F113C107F188
:1014400014C108F115C109F116C10AF117C10BF158
:1014500035C134F100C10CF101C10DF102C10EF131
:1014600003C10FF104C110F105C111F106C112F160
:1014700007C113F108C114F109C115F10AC116F130
:101480000BC117F134C135F101018E674FEF0AF03E
:101490008F674FEF0AF090674FEF0AF0916753EFB5
:1014A0000AF084EF0AF092C100F193C101F194C1F6
:1014B00002F195C103F10101010E046F000E056FE9
:1014C000000E066F000E076F82EC3BF000C192F138
:1014D00001C193F102C194F103C195F101010067CB
:1014E00079EF0AF0016779EF0AF0026779EF0AF005
:1014F000036784EF0AF08EC192F18FC193F190C11E
:1015000094F191C195F10F80109047C100F148C14D
:1015100001F149C102F14AC103F101010A0E046F50
:10152000000E056F000E066F000E076F82EC3BF099
:1015300003AF1080010154A7AAEF0AF00F9A0F9C85
:101540000F9E0101000E5E6F600E5F6F3D0E606FBB
:10155000080E616F47C100F148C101F149C102F1B4
:101560004AC103F10101140E046F050E056F000E50
:10157000066F000E076F82EC3BF003AFC3EF0AF07B
:10158000F288E8EF0AF0F2985E6B5F6B606B616B5C
:101590009A6B9B6B9C6B9D6B9E6B9F6BA06BA16B07
:1015A000A26BA36BA46BA56BA66BA76BA86BA96BB7
:1015B000AA6BAB6BAC6BAD6BAE6BAF6BB06BB16B67
:1015C000B26BB36BB46BB56BB66BB76BB86BB96B17
:1015D0000CC100F10DC101F10EC102F10FC103F107
:1015E00010C104F111C105F112C106F113C107F1D7
:1015F00014C108F115C109F116C10AF117C10BF1A7
:1016000035C134F104008BB40DEF0BF010AC0DEFCD
:101610000BF08B84109C0EEF0BF08B9407B465EFEE
:101620000BF007B065EF0BF01EC620F61FC621F6C3
:101630001CC61EF61DC61FF61AC61CF61BC61DF6D6
:1016400006C608F607C609F604C606F605C607F676
:1016500002C604F603C605F626C628F627C629F6EE
:1016600024C626F625C627F622C624F623C625F666
:101670000EC610F60FC611F60CC60EF60DC60FF606
:101680000AC60CF60BC60DF62EC630F62FC631F67E
:101690002CC62EF62DC62FF62AC62CF62BC62DF6F6
:1016A00016C618F617C619F614C616F615C617F696
:1016B00012C614F613C615F616B0E8EC3DF01EEC93
:1016C0003DF096EC3DF044EC3DF0077C07AC80EF3C
:1016D0000BF0C274C2B47AEF0BF0C3CFB7F5C4CF2E
:1016E000B8F50501D890B833B733D890B833B733CD
:1016F00081EF0BF0C3CF55F1C4CF56F181EF0BF062
:10170000C28207B4F3EF0BF047C14BF148C14CF173
:1017100049C14DF14AC14EF15EC162F15FC163F151
:1017200060C164F161C165F113A899EF0BF0138CEE
:1017300013989AC1BAF19BC1BBF19CC1BCF19DC188
:10174000BDF19EC1BEF19FC1BFF1A0C1C0F1A1C159
:10175000C1F1A2C1C2F1A3C1C3F1A4C1C4F1A5C129
:10176000C5F1A6C1C6F1A7C1C7F1A8C1C8F1A9C1F9
:10177000C9F1AAC1CAF1ABC1CBF1ACC1CCF1ADC1C9
:10178000CDF1AEC1CEF1AFC1CFF1B0C1D0F1B1C199
:10179000D1F1B2C1D2F1B3C1D3F1B4C1D4F1B5C169
:1017A000D5F1B6C1D6F1B7C1D7F1B8C1D8F1B9C139
:1017B000D9F1B7C5B9F5B8C5BAF5B9C5BBF5BAC55C
:1017C000BCF5010155515B2756515C23E86A5D2346
:1017D0000E2EF3EF0BF05CC157F15DC158F15B6B5E
:1017E0005C6B5D6B078EF5EF0BF002C0E0FF005005
:1017F00001C0D8FF1000A6B2FBEF0BF00CC0A9FF90
:101800000BC0A8FFA69EA69CA684F29E550EA76EAE
:10181000AA0EA76EA682F28EA694A6B20DEF0CF0C9
:101820000C2A1200A96EA69EA69CA680A8500C2A7F
:10183000120004012C0E826F88EC0FF097EC3CF044
:101840000C5012EC0CF0E8CF00F10C5012EC0CF044
:10185000E8CF01F101AF32EF0CF00101FF0E026F92
:10186000FF0E036F20EC3CF029673EEF0CF0040103
:10187000200E826F88EC0FF043EF0CF004012D0E68
:10188000826F88EC0FF02AEC3AF01200159415964E
:10189000076A0F6A106A116A126A136A176A0F01DF
:1018A0000D0EC16E860EC06E030EC26E0F01680E65
:1018B000896E130E926E080E8A6E8A6AF30E936E0C
:1018C000F10E936E8B6A900E946EC80E12EC0CF0B3
:1018D000E8CF26F000012650FE0AD8B47BEF0CF0CA
:1018E00000012650FD0AD8B480EF0CF00F0E276ED1
:1018F0008F0E286E09D00E0E276E8E0E286E04D025
:101900000D0E276E8D0E286E82EC3EF0C2EC3FF07D
:10191000F18EF19EFC0E12EC0CF0E8CF0BF00BA058
:1019200011800BA211820BA411840BA81188C90E7F
:1019300012EC0CF0E8CF1BF0CA0E12EC0CF0E8CF62
:101940001CF0CB0E12EC0CF0E8CF1DF0CC0E12EC1C
:101950000CF0E8CF1EF0FB0E12EC0CF0E8CF39F0E3
:10196000CE0E12EC0CF0E8CF14F0CD0E12EC0CF011
:10197000E8CF38F0206A216A0E6A01015B6B5C6B6C
:101980005D6B576B586BF29A0101476B486B496B63
:101990004A6B4B6B4C6B4D6B4E6B4F6B506B516B83
:1019A000526B456B466BD76AD66A0F01280ED56E0F
:1019B000F28A9D90B00ECD6E01015E6B5F6B606B25
:1019C000616B626B636B646B656B666B676B686B9B
:1019D000696B536B546BCF6ACE6A0F9A0F9C0F9E44
:1019E0009D80760ECA6E9D8202013C0E006FCC6A0D
:1019F000160E12EC0CF0E8CF00F1170E12EC0CF002
:101A0000E8CF01F1180E12EC0CF0E8CF02F1190E3C
:101A100012EC0CF0E8CF03F1010103AF2AEF0DF057
:101A200097EC3CF0160E0C6E00C10BF0FBEC0BF0CB
:101A3000170E0C6E01C10BF0FBEC0BF0180E0C6EC8
:101A400002C10BF0FBEC0BF0190E0C6E03C10BF096
:101A5000FBEC0BF000C18EF101C18FF102C190F1DE
:101A600003C191F100C192F101C193F102C194F15E
:101A700003C195F11A0E12EC0CF0E8CF00F11B0E29
:101A800012EC0CF0E8CF01F11C0E12EC0CF0E8CFD8
:101A900002F11D0E12EC0CF0E8CF03F1010103AFCF
:101AA00080EF0DF097EC3CF01A0E0C6E00C10BF0BD
:101AB000FBEC0BF01B0E0C6E01C10BF0FBEC0BF002
:101AC0001C0E0C6E02C10BF0FBEC0BF01D0E0C6E2D
:101AD00003C10BF0FBEC0BF01A0E12EC0CF0E8CF8C
:101AE00000F11B0E12EC0CF0E8CF01F11C0E12EC11
:101AF0000CF0E8CF02F11D0E12EC0CF0E8CF03F170
:101B000000C196F101C197F102C198F103C199F1A9
:101B1000240EAC6E900EAB6E240EAC6E080EB86E3A
:101B2000000EB06E1F0EAF6E0401806B816B0F0153
:101B3000900EAB6E0F019D8A0301806B816BC26BAF
:101B40008B9253EC43F053EC43F0880E12EC0CF004
:101B5000E8CF00F1890E12EC0CF0E8CF01F10101A1
:101B600001AFCBEF0DF097EC3CF0880E0C6E00C18E
:101B70000BF0FBEC0BF0890E0C6E01C10BF0FBECD3
:101B80000BF0880E12EC0CF0E8CF00F1890E12EC8D
:101B90000CF0E8CF01F100C140F601C141F602C1ED
:101BA00042F603C143F631EC47F031EC41F0200E30
:101BB00012EC0CF0E8CF2FF505012F51FF0AD8A445
:101BC000E9EF0DF02F6B200E0C6E2FC50BF0FBEC28
:101BD0000BF00501010E306F3C0E316F250E12EC3B
:101BE0000CF0E8CF00F1260E12EC0CF0E8CF01F17A
:101BF000270E12EC0CF0E8CF02F1280E12EC0CF0DC
:101C0000E8CF03F1010103AF20EF0EF097EC3CF0B9
:101C1000250E0C6E00C10BF0FBEC0BF0260E0C6ECB
:101C200001C10BF0FBEC0BF0270E0C6E02C10BF0A8
:101C3000FBEC0BF0280E0C6E03C10BF0FBEC0BF071
:101C400000C157F501C158F502C159F503C15AF554
:101C500000C15BF501C15CF502C15DF503C15EF534
:101C6000290E12EC0CF0E8CF5FF5050160515F5DC5
:101C7000D8A05FC560F5210E12EC0CF0E8CF00F1A2
:101C8000220E12EC0CF0E8CF01F1230E12EC0CF056
:101C9000E8CF02F1240E12EC0CF0E8CF03F10101C1
:101CA00003AF81EF0EF097EC3CF0210E0C6E00C1FB
:101CB0000BF0FBEC0BF0220E0C6E01C10BF0FBECF9
:101CC0000BF0230E0C6E02C10BF0FBEC0BF0240E9C
:101CD0000C6E03C10BF0FBEC0BF0210E12EC0CF0C0
:101CE000E8CF00F1220E12EC0CF0E8CF01F1230E48
:101CF00012EC0CF0E8CF02F1240E12EC0CF0E8CF5D
:101D000003F100C161F501C162F502C163F503C1D0
:101D100064F542EC40F05FEC3FF095EC3EF015903E
:101D2000C70E12EC0CF0E8CF00F1010100B19CEFFE
:101D30000EF015929DEF0EF0158281AAABEF0EF01A
:101D400015B4A6EF0EF01580ABEF0EF070EC47F077
:101D500015A0D9EF47F0E8EC3DF007900001F28EB6
:101D6000F28C12AE03D012BC6FEF21F007B0BCEFC3
:101D700037F00FB080EF30F010BE80EF30F012B8C7
:101D800080EF30F000011750010AD8B488EF27F037
:101D900081BAD3EF0EF000011750040AD8B42CEF2B
:101DA00024F0D9EF0EF000011750040AD8B4C4EFA4
:101DB00027F00301805181197F0BD8B4BCEF37F0B5
:101DC00013EE00F081517F0BE126812BE7CFE8FF76
:101DD000E00BD8B4BCEF37F023EE82F0C2513F0BDA
:101DE000D926E7CFDFFFC22BDF50780AD8A4BCEF9B
:101DF00037F0078092C100F193C101F194C102F163
:101E000095C103F10101040E046F000E056F000E71
:101E1000066F000E076F82EC3BF000AF19EF0FF07A
:101E20000101030E926F000E936F000E946F000E6F
:101E3000956F03018251720AD8B401EF30F08251DC
:101E4000520AD8B401EF30F08251750AD8B401EFCC
:101E500030F08251680AD8B49CEF0FF08251630AC7
:101E6000D8B476EF34F08251690AD8B4CEEF2AF0B4
:101E700082517A0AD8B4E1EF2BF08251490AD8B4E2
:101E80006DEF2AF08251500AD8B48BEF29F08251BD
:101E9000700AD8B4CEEF29F08251540AD8B4F9EFC1
:101EA00029F08251740AD8B43FEF2AF08251410AD6
:101EB000D8B4A1EF10F082514B0AD8B49EEF0FF0C6
:101EC00082516D0AD8B411EF15F082514D0AD8B481
:101ED0002AEF15F08251730AD8B431EF2FF08251F6
:101EE000530AD8B496EF2FF082514C0AD8B4C8EFF9
:101EF0001CF08251760AD8B4B9EF15F08251590A14
:101F0000D8B462EF14F012AE01D0128CADEF34F001
:101F1000040114EE00F080517F0BE12682C4E7FF3C
:101F2000802B120004010D0E826F88EC0FF00A0E58
:101F3000826F88EC0FF01200ABEF34F004014B0E0F
:101F4000826F88EC0FF004012C0E826F88EC0FF08A
:101F500081B802D038B630D003018351430AD8B4D7
:101F6000E3EF0FF003018351630AD8B4E5EF0FF0FC
:101F700003018351520AD8B4E7EF0FF003018351F4
:101F8000720AD8B4E9EF0FF003018351470AD8B4BD
:101F9000EBEF0FF003018351670AD8B4EDEF0FF0B8
:101FA00003018351540AD8B4EFEF0FF003018351BA
:101FB000740AD8B45FEF10F003018351550AD8B406
:101FC000F1EF0FF083D038807BD0389079D0388211
:101FD00077D0389275D0388473D0389471D03886E1
:101FE0006FD084C330F185C331F186C332F187C32A
:101FF00033F10101296BE5EC3CF05CEC3CF000C1F5
:1020000004F101C105F102C106F103C107F1D8ECE9
:102010003CF0200EF86EF76AF66A0900F5CF2CF155
:102020000900F5CF2DF10900F5CF2EF10900F5CF0C
:102030002FF10900F5CF30F10900F5CF31F109009A
:10204000F5CF32F10900F5CF33F10101296BE5EC51
:102050003CF05CEC3CF082EC3BF00101006738EFB7
:1020600010F0016738EF10F0026738EF10F00367E7
:1020700001D025D004014E0E826F88EC0FF00401D0
:102080006F0E826F88EC0FF004014D0E826F88ECAA
:102090000FF00401610E826F88EC0FF00401740EE2
:1020A000826F88EC0FF00401630E826F88EC0FF0F2
:1020B0000401680E826F88EC0FF0ABEF34F03896B5
:1020C000CD0E0C6E38C00BF0FBEC0BF0CD0E12EC0D
:1020D0000CF0E8CF38F038B006D00401630E826F00
:1020E00088EC0FF005D00401430E826F88EC0FF0EE
:1020F00038B206D00401720E826F88EC0FF005D062
:102100000401520E826F88EC0FF038B406D004013F
:10211000670E826F88EC0FF005D00401470E826FC6
:1021200088EC0FF038B606D00401740E826F88EC8C
:102130000FF005D00401540E826F88EC0FF0ABEF66
:1021400034F00401410E826F88EC0FF003018351DB
:10215000310AD8B482EF13F003018351320AD8B4A4
:10216000B2EF12F003018351330AD8B43BEF12F0FF
:1021700003018351340AD8B42BEF11F003018351CA
:10218000350AD8B4CBEF10F004013F0E826F88EC13
:102190000FF0ABEF34F003018451300AD8B4F1EF03
:1021A00010F003018451310AD8B4F4EF10F00301A8
:1021B0008451650AD8B4E5EF10F003018451640A34
:1021C000D8B4E8EF10F0F5EF10F03990E9EF10F027
:1021D0003980FB0E0C6E39C00BF0FBEC0BF0F5EF09
:1021E00010F08B90F5EF10F08B800401350E826FAC
:1021F00088EC0FF004012C0E826F88EC0FF08BB08E
:1022000009EF11F00401300E826F88EC0FF00EEF31
:1022100011F00401310E826F88EC0FF004012C0ED6
:10222000826F88EC0FF0FB0E12EC0CF0E8CF39F067
:1022300039A022EF11F00401640E826F88EC0FF0D8
:1022400027EF11F00401650E826F88EC0FF029EF83
:1022500011F0ABEF34F0CC0E12EC0CF0E8CF0BF039
:1022600004012C0E826F88EC0FF003018451310AB7
:10227000D8B44FEF11F003018451300AD8B451EFB4
:1022800011F0030184514D0AD8B45BEF11F0030142
:102290008451540AD8B462EF11F079EF11F08A84B6
:1022A00001D08A940BAE04D00BAC02D00BBA21D073
:1022B000E00E0B1218D01F0E0B168539E844E00B08
:1022C0000B1211D0E00E0B16D8EC3CF085C332F1A6
:1022D00086C333F10101296BE5EC3CF05CEC3CF08A
:1022E00000511F0B0B12CC0E0C6E0BC00BF0FBEC55
:1022F0000BF00401340E826F88EC0FF004012C0EF9
:10230000826F88EC0FF0CC0E12EC0CF0E8CF1EF0D0
:102310008AB406D00401300E826F88EC0FF005D02D
:102320000401310E826F88EC0FF004012C0E826FD5
:1023300088EC0FF01E38E840070BE8CF82F4040168
:10234000300E822788EC0FF004012C0E826F88EC8F
:102350000FF097EC3CF01E501F0BE8CF00F120EC83
:102360003CF032C182F40401300E822788EC0FF079
:1023700033C182F40401300E822788EC0FF004018F
:102380002C0E826F88EC0FF097EC3CF032C000F11D
:1023900000AF0BD0FF0E016FFF0E026FFF0E036F39
:1023A00004012D0E826F88EC0FF020EC3CF031C15F
:1023B00082F40401300E822788EC0FF032C182F4DF
:1023C0000401300E822788EC0FF033C182F404013F
:1023D000300E822788EC0FF004012C0E826F88ECFF
:1023E0000FF097EC3CF031C000F120EC3CF031C133
:1023F00082F40401300E822788EC0FF032C182F49F
:102400000401300E822788EC0FF033C182F40401FE
:10241000300E822788EC0FF004012C0E826F88ECBE
:102420000FF097EC3CF033C000F100AF0BD0FF0E83
:10243000016FFF0E026FFF0E036F04012D0E826FFE
:1024400088EC0FF020EC3CF031C182F40401300E36
:10245000822788EC0FF032C182F40401300E82270B
:1024600088EC0FF033C182F40401300E822788EC2F
:102470000FF0ABEF34F0CB0E12EC0CF0E8CF0BF01A
:1024800004012C0E826F88EC0FF003018451450A81
:10249000D8B45FEF12F003018451440AD8B462EF5C
:1024A00012F003018451300AD8B465EF12F0030131
:1024B0008451310AD8B469EF12F074EF12F00B9E18
:1024C0006EEF12F00B8E6EEF12F0FC0E0B166EEF2D
:1024D00012F0FC0E0B160B806EEF12F0CB0E0C6E92
:1024E0000BC00BF0FBEC0BF00401330E826F88EC99
:1024F0000FF004012C0E826F88EC0FF0CB0E12EC63
:102500000CF0E8CF1DF01DBE8DEF12F00401450E5A
:10251000826F88EC0FF092EF12F00401440E826F8C
:1025200088EC0FF004012C0E826F88EC0FF0040190
:10253000300E826F88EC0FF004012C0E826F88EC55
:102540000FF01DB0ABEF12F00401300E826F88EC7B
:102550000FF0B0EF12F00401310E826F88EC0FF033
:10256000ABEF34F0CA0E12EC0CF0E8CF0BF0040124
:102570002C0E826F88EC0FF003018451450AD8B409
:10258000EEEF12F003018451440AD8B4F1EF12F0D7
:10259000030184514D0AD8B4FAEF12F003018451BB
:1025A000410AD8B4F4EF12F003018451460AD8B4BA
:1025B000F7EF12F003018451560AD8B402EF13F07A
:1025C00003018451500AD8B40DEF13F00301845174
:1025D000520AD8B410EF13F019EF13F00B9E13EF5B
:1025E00013F00B8E13EF13F00B9C13EF13F00B8C07
:1025F00013EF13F0FC0E0B1685C3E8FF030B0B1251
:1026000013EF13F0C70E0B1685C3E8FF070BE84660
:10261000E846E8460B1213EF13F00B8413EF13F0A8
:102620000B9413EF13F0CA0E0C6E0BC00BF0FBEC07
:102630000BF0CA0E12EC0CF0E8CF1CF00401320EC5
:10264000826F88EC0FF004012C0E826F88EC0FF083
:102650001CBE32EF13F00401450E826F88EC0FF0C0
:1026600037EF13F00401440E826F88EC0FF0040181
:102670002C0E826F88EC0FF01CC0E8FF030BE8CF34
:1026800082F40401300E822788EC0FF004012C0E36
:10269000826F88EC0FF01CBC55EF13F00401410E63
:1026A000826F88EC0FF05AEF13F00401460E826F30
:1026B00088EC0FF004012C0E826F88EC0FF01CC028
:1026C000E8FF380BE842E842E842E8CF82F4040130
:1026D000300E822788EC0FF004012C0E826F88ECFC
:1026E0000FF01CB47BEF13F00401520E826F88ECE4
:1026F0000FF080EF13F00401500E826F88EC0FF0A2
:10270000ABEF34F0C90E12EC0CF0E8CF0BF0040183
:102710002C0E826F88EC0FF003018451450AD8B467
:10272000A0EF13F003018451440AD8B4A3EF13F0CF
:10273000030184514D0AD8B4A6EF13F0B4EF13F09F
:102740000B9EAEEF13F00B8EAEEF13F0F80E0B16E0
:1027500085C3E8FF070B0B12AEEF13F0C90E0C6E2A
:102760000BC00BF0FBEC0BF00401310E826F88EC18
:102770000FF004012C0E826F88EC0FF0C90E12ECE2
:102780000CF0E8CF1BF01BBE06D00401450E826F93
:1027900088EC0FF005D00401440E826F88EC0FF036
:1027A00004012C0E826F88EC0FF01BC0E8FF070BB2
:1027B000E8CF82F40401300E822788EC0FF0040188
:1027C0002C0E826F88EC0FF0078097EC3CF02DC048
:1027D000E8FF003B00430043030B20EC3CF033C117
:1027E00082F40401300E822788EC0FF004012C0ED5
:1027F000826F88EC0FF097EC3CF02DC001F1019F47
:10280000019D2EC000F1010120EC3CF02FC182F4AB
:102810000401300E822788EC0FF030C182F40401ED
:10282000300E822788EC0FF031C182F40401300EA3
:10283000822788EC0FF032C182F40401300E822727
:1028400088EC0FF033C182F40401300E822788EC4B
:102850000FF004012C0E826F88EC0FF097EC3CF027
:102860002FC001F130C000F1D89001330033D8906F
:1028700001330033010120EC3CF02FC182F404014C
:10288000300E822788EC0FF030C182F40401300E44
:10289000822788EC0FF031C182F40401300E8227C8
:1028A00088EC0FF032C182F40401300E822788ECEC
:1028B0000FF033C182F40401300E822788EC0FF050
:1028C000ABEF34F0FC0E12EC0CF0E8CF0BF0030190
:1028D0008351520AD8B499EF14F003018351720A5C
:1028E000D8B49CEF14F003018351500AD8B49FEF81
:1028F00014F003018351700AD8B4A2EF14F003015D
:102900008351550AD8B4A5EF14F003018351750A19
:10291000D8B4A8EF14F003018351430AD8B4B1EF3F
:1029200014F003018351630AD8B4B4EF14F0BDEF7F
:1029300014F00B90B7EF14F00B80B7EF14F00B927C
:10294000B7EF14F00B82B7EF14F00B94B7EF14F05D
:102950000B84B7EF14F00B96B7EF14F00B86B7EFBC
:1029600014F00B98B7EF14F00B88B7EF14F0FC0ECF
:102970000C6E0BC00BF0FBEC0BF00401590E826FD8
:1029800088EC0FF01190119211941198FC0E12EC3A
:102990000CF0E8CF0BF00BA011800BA211820BA45E
:1029A00011840BA8118811A0DDEF14F00401520E60
:1029B000826F88EC0FF0E2EF14F00401720E826F68
:1029C00088EC0FF011A8ECEF14F00401430E826FB5
:1029D00088EC0FF0F1EF14F00401630E826F88ECC5
:1029E0000FF011A2FBEF14F00401500E826F88EC7F
:1029F0000FF000EF15F00401700E826F88EC0FF0FD
:102A000011A40AEF15F00401550E826F88EC0FF047
:102A10000FEF15F00401750E826F88EC0FF0ABEF2D
:102A200034F004016D0E826F88EC0FF003018351C6
:102A3000300AD8B469EF15F003018351310AD8B4D4
:102A40007CEF15F003018351320AD8B48FEF15F0F3
:102A5000ADEF34F004014D0E826F88EC0FF0D8EC2E
:102A60003CF084C331F185C332F186C333F10101F7
:102A7000296BE5EC3CF05CEC3CF003018351300A3F
:102A8000D8B451EF15F003018351310AD8B459EF8E
:102A900015F003018351320AD8B461EF15F0ADEFA0
:102AA00034F0FD0E0C6E00C10BF0FBEC0BF069EF87
:102AB00015F0FE0E0C6E00C10BF0FBEC0BF07CEF82
:102AC00015F0FF0E0C6E00C10BF0FBEC0BF08FEF5E
:102AD00015F00401300E826F88EC0FF004012C0E0B
:102AE000826F88EC0FF097EC3CF0FD0E12EC0CF0CE
:102AF000E8CF00F1A0EF15F00401310E826F88ECF1
:102B00000FF004012C0E826F88EC0FF097EC3CF074
:102B1000FE0E12EC0CF0E8CF00F1A0EF15F004016E
:102B2000320E826F88EC0FF097EC3CF004012C0E13
:102B3000826F88EC0FF0FF0E12EC0CF0E8CF00F182
:102B400020EC3CF031C182F40401300E822788EC85
:102B50000FF032C182F40401300E822788EC0FF0AE
:102B600033C182F40401300E822788EC0FF0ABEF02
:102B700034F003018351300AD8B464EF17F0030135
:102B80008351310AD8B4C3EF17F003018351320ADD
:102B9000D8B478EF19F003018351330AD8B42DEF7C
:102BA0001BF003018351340AD8B4D3EF1BF00301A7
:102BB0008351350AD8B4BBEF1CF003018351730A6B
:102BC000D8B446EF16F003018351760AD8B448EF23
:102BD00016F003018351740AD8B433EF16F00301E1
:102BE0008351540AD8B4F8EF15F0D8A4ADEF34F0FF
:102BF0000401760E826F88EC0FF00401540E826F90
:102C000088EC0FF007840001880E0C6ED8EC3CF0C5
:102C10002981030184512D0AD8B411EF16F0010166
:102C2000299185C32FF186C330F187C331F188C361
:102C300032F189C333F1E5EC3CF05CEC3CF000C1CF
:102C40000BF0FBEC0BF001C10BF0FBEC0BF0880E72
:102C500012EC0CF0E8CF40F6890E12EC0CF0E8CF45
:102C600041F63EEF16F00401760E826F88EC0FF00D
:102C70000401740E826F88EC0FF007840001880E47
:102C80000C6E19EC0CF0079438EF28F046EC16F0B7
:102C90000401760E826F88EC0FF00401760E826FCD
:102CA00088EC0FF00784DAEC38F004012C0E826F08
:102CB00088EC0FF00101036B026B3BC601F13AC6D1
:102CC00000F101AF69EF16F00101FF0E026FFF0E78
:102CD000036F20EC3CF0296770EF16F075EF16F0EB
:102CE00004012D0E826F88EC0FF02FC182F40401D5
:102CF000300E822788EC0FF030C182F40401300ED0
:102D0000822788EC0FF031C182F40401300E822753
:102D100088EC0FF032C182F40401300E822788EC77
:102D20000FF033C182F40401300E822788EC0FF0DB
:102D300004012C0E826F88EC0FF00101036B026B13
:102D40003DC601F13CC600F101AFACEF16F0010148
:102D5000FF0E026FFF0E036F20EC3CF02967B3EF0C
:102D600016F0B8EF16F004012D0E826F88EC0FF00C
:102D70002FC182F40401300E822788EC0FF030C19D
:102D800082F40401300E822788EC0FF031C182F406
:102D90000401300E822788EC0FF032C182F4040166
:102DA000300E822788EC0FF033C182F40401300E1C
:102DB000822788EC0FF004012C0E826F88EC0FF054
:102DC0000101036B026B3FC601F13EC600F101AF8A
:102DD000EFEF16F00101FF0E026FFF0E036F20EC04
:102DE0003CF02967F6EF16F0FBEF16F004012D0E0C
:102DF000826F88EC0FF02FC182F40401300E82271D
:102E000088EC0FF030C182F40401300E822788EC88
:102E10000FF031C182F40401300E822788EC0FF0EC
:102E200032C182F40401300E822788EC0FF033C1E6
:102E300082F40401300E822788EC0FF004012C0E7E
:102E4000826F88EC0FF00101036B026B37C601F152
:102E500036C600F101AF32EF17F00101FF0E026F2D
:102E6000FF0E036F20EC3CF0296739EF17F03EEFBF
:102E700017F004012D0E826F88EC0FF02FC182F441
:102E80000401300E822788EC0FF030C182F4040177
:102E9000300E822788EC0FF031C182F40401300E2D
:102EA000822788EC0FF032C182F40401300E8227B1
:102EB00088EC0FF033C182F40401300E822788ECD5
:102EC0000FF0079438EF28F00401760E826F88EC3B
:102ED0000FF00401300E826F88EC0FF004012C0E0D
:102EE000826F88EC0FF097EC3CF000C600F101C651
:102EF00001F120EC3CF02AC182F40401300E82275B
:102F000088EC0FF02BC182F40401300E822788EC8C
:102F10000FF02CC182F40401300E822788EC0FF0F0
:102F20002DC182F40401300E822788EC0FF02EC1EF
:102F300082F40401300E822788EC0FF02FC182F456
:102F40000401300E822788EC0FF030C182F40401B6
:102F5000300E822788EC0FF031C182F40401300E6C
:102F6000822788EC0FF032C182F40401300E8227F0
:102F700088EC0FF033C182F40401300E822788EC14
:102F80000FF038EF28F00401760E826F88EC0FF016
:102F90000401310E826F88EC0FF007840101036B8E
:102FA000026B02C600F103C601F101AFDCEF17F0BE
:102FB000FF0E026FFF0E036F0101076B066B04C665
:102FC00004F105C605F105AFEAEF17F0FF0E066F35
:102FD000FF0E076F87EC3BF00101076B066B06C61F
:102FE00004F107C605F105AFFAEF17F0FF0E066F03
:102FF000FF0E076F87EC3BF00101076B066B08C6FD
:1030000004F109C605F105AF0AEF18F0FF0E066FCF
:10301000FF0E076F87EC3BF0D890010103330233BA
:1030200001330033D89001010333023301330033FD
:1030300004012C0E826F88EC0FF00101036B026B10
:1030400001C101F100C100F101AF2CEF18F0010145
:10305000FF0E026FFF0E036F20EC3CF0296733EF89
:1030600018F038EF18F004012D0E826F88EC0FF085
:103070002FC182F40401300E822788EC0FF030C19A
:1030800082F40401300E822788EC0FF031C182F403
:103090000401300E822788EC0FF032C182F4040163
:1030A000300E822788EC0FF033C182F40401300E19
:1030B000822788EC0FF00101036B026B0AC600F156
:1030C0000BC601F101AF69EF18F0FF0E026FFF0EA2
:1030D000036F0101076B066B0CC604F10DC605F109
:1030E00005AF77EF18F0FF0E066FFF0E076F87EC46
:1030F0003BF00101076B066B0EC604F10FC605F12C
:1031000005AF87EF18F0FF0E066FFF0E076F87EC15
:103110003BF00101076B066B10C604F111C605F107
:1031200005AF97EF18F0FF0E066FFF0E076F87ECE5
:103130003BF0D89001010333023301330033D890C0
:103140000101033302330133003304012C0E826F7B
:1031500088EC0FF00101036B026B01C101F100C1AA
:1031600000F101AFB9EF18F00101FF0E026FFF0E81
:10317000036F20EC3CF02967C0EF18F0C5EF18F0A2
:1031800004012D0E826F88EC0FF02FC182F4040130
:10319000300E822788EC0FF030C182F40401300E2B
:1031A000822788EC0FF031C182F40401300E8227AF
:1031B00088EC0FF032C182F40401300E822788ECD3
:1031C0000FF033C182F40401300E822788EC0FF037
:1031D0000101036B026B12C600F113C601F101AFCE
:1031E000F6EF18F0FF0E026FFF0E036F0101076B81
:1031F000066B14C604F115C605F105AF04EF19F00E
:10320000FF0E066FFF0E076F87EC3BF00101076BA7
:10321000066B16C604F117C605F105AF14EF19F0D9
:10322000FF0E066FFF0E076F87EC3BF00101076B87
:10323000066B18C604F119C605F105AF24EF19F0A5
:10324000FF0E066FFF0E076F87EC3BF0D890010171
:103250000333023301330033D890010103330233C7
:103260000133003304012C0E826F88EC0FF0010152
:10327000036B026B01C101F100C100F101AF46EF28
:1032800019F00101FF0E026FFF0E036F20EC3CF0FE
:1032900029674DEF19F052EF19F004012D0E826FDE
:1032A00088EC0FF02FC182F40401300E822788ECE5
:1032B0000FF030C182F40401300E822788EC0FF049
:1032C00031C182F40401300E822788EC0FF032C144
:1032D00082F40401300E822788EC0FF033C182F4AF
:1032E0000401300E822788EC0FF0079438EF28F0A5
:1032F0000401760E826F88EC0FF00401320E826FAB
:1033000088EC0FF007840101036B026B1AC600F111
:103310001BC601F101AF91EF19F0FF0E026FFF0E16
:10332000036F0101076B066B1CC604F11DC605F196
:1033300005AF9FEF19F0FF0E066FFF0E076F87ECCA
:103340003BF00101076B066B1EC604F11FC605F1B9
:1033500005AFAFEF19F0FF0E066FFF0E076F87EC9A
:103360003BF00101076B066B20C604F121C605F195
:1033700005AFBFEF19F0FF0E066FFF0E076F87EC6A
:103380003BF0D89001010333023301330033D8906E
:103390000101033302330133003304012C0E826F29
:1033A00088EC0FF00101036B026B01C101F100C158
:1033B00000F101AFE1EF19F00101FF0E026FFF0E06
:1033C000036F20EC3CF02967E8EF19F0EDEF19F0FE
:1033D00004012D0E826F88EC0FF02FC182F40401DE
:1033E000300E822788EC0FF030C182F40401300ED9
:1033F000822788EC0FF031C182F40401300E82275D
:1034000088EC0FF032C182F40401300E822788EC80
:103410000FF033C182F40401300E822788EC0FF0E4
:103420000101036B026B22C600F123C601F101AF5B
:103430001EEF1AF0FF0E026FFF0E036F0101076B04
:10344000066B24C604F125C605F105AF2CEF1AF072
:10345000FF0E066FFF0E076F87EC3BF00101076B55
:10346000066B26C604F127C605F105AF3CEF1AF03E
:10347000FF0E066FFF0E076F87EC3BF00101076B35
:10348000066B28C604F129C605F105AF4CEF1AF00A
:10349000FF0E066FFF0E076F87EC3BF0D89001011F
:1034A0000333023301330033D89001010333023375
:1034B0000133003304012C0E826F88EC0FF0010100
:1034C000036B026B01C101F100C100F101AF6EEFAE
:1034D0001AF00101FF0E026FFF0E036F20EC3CF0AB
:1034E000296775EF1AF07AEF1AF004012D0E826F3A
:1034F00088EC0FF02FC182F40401300E822788EC93
:103500000FF030C182F40401300E822788EC0FF0F6
:1035100031C182F40401300E822788EC0FF032C1F1
:1035200082F40401300E822788EC0FF033C182F45C
:103530000401300E822788EC0FF00101036B026B4F
:103540002AC600F12BC601F101AFABEF1AF0FF0E56
:10355000026FFF0E036F0101076B066B2CC604F1AF
:103560002DC605F105AFB9EF1AF0FF0E066FFF0E7D
:10357000076F87EC3BF00101076B066B2EC604F169
:103580002FC605F105AFC9EF1AF0FF0E066FFF0E4B
:10359000076F87EC3BF00101076B066B30C604F147
:1035A00031C605F105AFD9EF1AF0FF0E066FFF0E19
:1035B000076F87EC3BF0D8900101033302330133EE
:1035C0000033D89001010333023301330033040187
:1035D0002C0E826F88EC0FF00101036B026B01C1AE
:1035E00001F100C100F101AFFBEF1AF00101FF0E84
:1035F000026FFF0E036F20EC3CF0296702EF1BF017
:1036000007EF1BF004012D0E826F88EC0FF02FC125
:1036100082F40401300E822788EC0FF030C182F46E
:103620000401300E822788EC0FF031C182F40401CE
:10363000300E822788EC0FF032C182F40401300E84
:10364000822788EC0FF033C182F40401300E822708
:1036500088EC0FF0079438EF28F00401760E826FA3
:1036600088EC0FF00401330E826F88EC0FF0040138
:103670002C0E826F88EC0FF085C382F488EC0FF07B
:10368000640E0D6E03018551320A02E16A0E0D6E61
:1036900003018551330A02E1700E0D6E030185515D
:1036A000340A02E1760E0D6E03018551350A02E1FE
:1036B0007C0E0D6E03018551360A02E1820E0D6EFD
:1036C00003018651780A65E00DC00CF0D8EC3CF09F
:1036D0002981030187512D0AD8B471EF1BF0010134
:1036E000299188C32FF189C330F18AC331F18BC38B
:1036F00032F18CC333F1E5EC3CF05CEC3CF000C102
:103700000BF0FBEC0BF001C10BF0FBEC0BF0D8EC79
:103710003CF0298103018E512D0AD8B492EF1BF0A1
:10372000010129918FC32FF190C330F191C331F181
:1037300092C332F193C333F1E5EC3CF05CEC3CF026
:1037400000C10BF0FBEC0BF001C10BF0FBEC0BF03C
:10375000D8EC3CF02981030195512D0AD8B4B3EF80
:103760001BF00101299196C32FF197C330F198C343
:1037700031F199C332F19AC333F1E5EC3CF05CECE2
:103780003CF000C10BF0FBEC0BF001C10BF0FBECCB
:103790000BF00DC00CF019EC0CF019EC0CF019EC5E
:1037A0000CF038EF28F00401760E826F88EC0FF0F1
:1037B0000401340E826F88EC0FF003018451780A03
:1037C000D8B4ABEF1CF03E0E0C6ED8EC3CF0298167
:1037D000030185512D0AD8B4F0EF1BF001012991A6
:1037E00086C32FF187C330F188C331F189C332F129
:1037F0008AC333F1E5EC3CF05CEC3CF000C10BF02B
:10380000FBEC0BF001C10BF0FBEC0BF0D8EC3CF047
:10381000298103018C512D0AD8B411EF1CF001014C
:1038200029918DC32FF18EC330F18FC331F190C335
:1038300032F191C333F1E5EC3CF05CEC3CF000C1BB
:103840000BF0FBEC0BF001C10BF0FBEC0BF0D8EC38
:103850003CF02981030193512D0AD8B432EF1CF0BA
:103860000101299194C32FF195C330F196C331F131
:1038700097C332F198C333F1E5EC3CF05CEC3CF0DB
:1038800000C10BF0FBEC0BF001C10BF0FBEC0BF0FB
:10389000D8EC3CF0298103019A512D0AD8B453EF9A
:1038A0001CF0010129919BC32FF19CC330F19DC3F2
:1038B00031F19EC332F19FC333F1E5EC3CF05CEC97
:1038C0003CF000C10BF0FBEC0BF001C10BF0FBEC8A
:1038D0000BF0D8EC3CF029810301A1512D0AD8B49A
:1038E00074EF1CF001012991A2C32FF1A3C330F1A1
:1038F000A4C331F1A5C332F1A6C333F1E5EC3CF02A
:103900005CEC3CF000C10BF0FBEC0BF001C10BF0E8
:10391000FBEC0BF0D8EC3CF029810301A8512D0AF7
:10392000D8B495EF1CF001012991A9C32FF1AAC3C6
:1039300030F1ABC331F1ACC332F1ADC333F1E5ECDF
:103940003CF05CEC3CF000C10BF0FBEC0BF001C177
:103950000BF0FBEC0BF03E0E0C6E19EC0CF019ECBE
:103960000CF019EC0CF019EC0CF019EC0CF019EC53
:103970000CF038EF28F016800401760E826F88EC88
:103980000FF00401350E826F88EC0FF038EF28F04D
:1039900003018351300AD8B41CEF22F00301835194
:1039A000310AD8B45AEF23F003018351320AD8B454
:1039B000C8EF23F003018351330AD8B4D8EF23F0C2
:1039C00003018351340AD8B433EF24F00301835147
:1039D000350AD8B4DCEF27F003018351360AD8B496
:1039E0000AEF28F003018351370AD8B4F4EF1FF02F
:1039F00003018351380AD8B492EF20F003018351B8
:103A0000440AD8B420EF1EF003018351640AD8B4ED
:103A100040EF1EF003018351460AD8B4E1EF26F0CF
:103A2000030183514D0AD8B46DEF1EF00301835199
:103A30006D0AD8B487EF1EF0030183515A0AD8B437
:103A4000D4EF22F003018351490AD8B40AEF29F0D8
:103A500003018351500AD8B43CEF28F0030183518D
:103A6000540AD8B4B5EF28F003018351630AD8B4DF
:103A7000A7EF1EF003018351430AD8B49FEF1FF054
:103A800003018351730AD8B4A5EF1EF003018351DB
:103A9000610AD8B46DEF1DF003018351650AD8B4F3
:103AA0006CEF22F003018351450AD8B47AEF22F07B
:103AB00003018351620AD8B488EF22F003018351D5
:103AC000420AD8B496EF22F003018351760AD8B4A3
:103AD000A4EF22F0D8A4ADEF34F004014C0E826FB5
:103AE00088EC0FF00401610E826F88EC0FF05FEC40
:103AF0003FF004012C0E826F88EC0FF097EC3CF045
:103B0000AFC500F1010120EC3CF031C182F40401A9
:103B1000300E822788EC0FF032C182F40401300E9F
:103B2000822788EC0FF033C182F40401300E822723
:103B300088EC0FF004012C0E826F88EC0FF097ECEC
:103B40003CF0B0C500F1010120EC3CF031C182F441
:103B50000401300E822788EC0FF032C182F4040198
:103B6000300E822788EC0FF033C182F40401300E4E
:103B7000822788EC0FF004012C0E826F88EC0FF086
:103B800097EC3CF0B1C500F1010120EC3CF031C1F3
:103B900082F40401300E822788EC0FF032C182F4E7
:103BA0000401300E822788EC0FF033C182F4040147
:103BB000300E822788EC0FF004012C0E826F88EC07
:103BC0000FF097EC3CF0B2C500F1010120EC3CF0A5
:103BD00031C182F40401300E822788EC0FF032C12B
:103BE00082F40401300E822788EC0FF033C182F496
:103BF0000401300E822788EC0FF004012C0E826F36
:103C000088EC0FF097EC3CF0B6C500F1010120EC18
:103C10003CF031C182F40401300E822788EC0FF0B1
:103C200032C182F40401300E822788EC0FF033C1D8
:103C300082F40401300E822788EC0FF038EF28F070
:103C400003018451300AD8B42CEF1EF003018451D3
:103C5000310AD8B430EF1EF01592159631EF1EF0F0
:103C60001582C70E12EC0CF0E8CF00F101010081C3
:103C700015A20091C70E0C6E00C10BF0FBEC0BF00F
:103C8000C70E12EC0CF0E8CF00F1010100B14CEFCF
:103C90001EF015924DEF1EF0158204014C0E826F3E
:103CA00088EC0FF00401640E826F88EC0FF00401C1
:103CB0002C0E826F88EC0FF015B266EF1EF0040137
:103CC000300E826F88EC0FF06BEF1EF00401310EA6
:103CD000826F88EC0FF0ABEF34F0D8EC3CF084C38B
:103CE00033F1E5EC3CF05CEC3CF0200E0C6E00C1D6
:103CF0000BF0FBEC0BF000C12FF505012F51000A72
:103D000006E005012F51010A02E0C2EC3FF0040178
:103D10004C0E826F88EC0FF004014D0E826F88EC20
:103D20000FF004012C0E826F88EC0FF097EC3CF042
:103D30002FC500F120EC3CF033C182F40401300EB9
:103D4000822788EC0FF038EF28F0D9EF47F0040114
:103D50004C0E826F88EC0FF00401630E826F88ECCA
:103D60000FF095EC3EF004012C0E826F88EC0FF002
:103D7000BCEC1EF038EF28F097EC3CF0B5C500F134
:103D80000101003B0F0E001720EC3CF033C182F420
:103D90000401300E822788EC0FF0B5C500F1010157
:103DA0000F0E0101001720EC3CF033C182F4040136
:103DB000300E822788EC0FF004012D0E826F88EC04
:103DC0000FF0B4C500F10101003B0F0E001720EC0D
:103DD0003CF033C182F40401300E822788EC0FF0EE
:103DE000B4C500F101010F0E0101001720EC3CF0F9
:103DF00033C182F40401300E822788EC0FF00401F5
:103E00002D0E826F88EC0FF0B3C500F10101003B6D
:103E10000F0E001720EC3CF033C182F40401300E89
:103E2000822788EC0FF0B3C500F101010F0E0101EC
:103E3000001720EC3CF033C182F40401300E8227DD
:103E400088EC0FF00401200E826F88EC0FF0B2C5F1
:103E500000F10F0E0101001720EC3CF033C182F499
:103E60000401300E822788EC0FF00401200E826FCF
:103E700088EC0FF0B1C500F101010101003B0F0E0C
:103E8000001720EC3CF033C182F40401300E82278D
:103E900088EC0FF0B1C500F101010F0E0101001710
:103EA00020EC3CF033C182F40401300E822788EC10
:103EB0000FF004013A0E826F88EC0FF0B0C500F1EC
:103EC0000101003B0F0E001720EC3CF033C182F4DF
:103ED0000401300E822788EC0FF0B0C500F101011B
:103EE0000F0E0101001720EC3CF033C182F40401F5
:103EF000300E822788EC0FF004013A0E826F88ECB6
:103F00000FF0AFC500F10101003B0F0E001720ECD0
:103F10003CF033C182F40401300E822788EC0FF0AC
:103F2000AFC500F101010F0E001720EC3CF033C1CA
:103F300082F40401300E822788EC0FF0120084C353
:103F4000E8FF0F0BE83AE8CFB5F585C3E8FF0F0BA4
:103F50000501B51387C3E8FF0F0BE83AE8CFB4F5C6
:103F600088C3E8FF0F0B0501B4138AC3E8FF0F0BEA
:103F7000E83AE8CFB3F58BC3E8FF0F0B0501B313A5
:103F80008DC3E8FF0F0BE8CFB2F58FC3E8FF0F0B2F
:103F9000E83AE8CFB1F590C3E8FF0F0B0501B11384
:103FA00092C3E8FF0F0BE83AE8CFB0F593C3E8FF00
:103FB0000F0B0501B01395C3E8FF0F0BE83AE8CFEC
:103FC000AFF596C3E8FF0F0B0501AF1301EC3FF00F
:103FD00004014C0E826F88EC0FF00401430E826FD7
:103FE00088EC0FF0B1EF1EF0078404014C0E826FD5
:103FF00088EC0FF00401370E826F88EC0FF004019B
:104000002C0E826F88EC0FF005012E51130A06E08A
:1040100005012E51170A0DE08FEF20F00101000E6F
:10402000006F000E016F100E026F000E036F22EF83
:1040300020F00101000E006F000E016F000E026FF4
:10404000010E036F20EC3CF02AC182F40401300E13
:10405000822788EC0FF02BC182F40401300E8227F6
:1040600088EC0FF02CC182F40401300E822788EC1A
:104070000FF02DC182F40401300E822788EC0FF07E
:104080002EC182F40401300E822788EC0FF02FC17C
:1040900082F40401300E822788EC0FF030C182F4E4
:1040A0000401300E822788EC0FF031C182F4040144
:1040B000300E822788EC0FF032C182F40401300EFA
:1040C000822788EC0FF033C182F40401300E82277E
:1040D00088EC0FF004012C0E826F88EC0FF00101C8
:1040E000200E006F000E016F000E026F000E036FB6
:1040F00020EC3CF031C182F40401300E822788ECC0
:104100000FF032C182F40401300E822788EC0FF0E8
:1041100033C182F40401300E822788EC0FF007943B
:1041200038EF28F00501216B226B236B246B04010F
:104130004C0E826F88EC0FF00401380E826F88EC11
:104140000FF004012C0E826F88EC0FF00101200E9D
:10415000006F000E016F000E026F000E036F20EC67
:104160003CF02AC182F40401300E822788EC0FF063
:104170002BC182F40401300E822788EC0FF02CC191
:1041800082F40401300E822788EC0FF02DC182F4F6
:104190000401300E822788EC0FF02EC182F4040156
:1041A000300E822788EC0FF02FC182F40401300E0C
:1041B000822788EC0FF030C182F40401300E822790
:1041C00088EC0FF031C182F40401300E822788ECB4
:1041D0000FF032C182F40401300E822788EC0FF018
:1041E00033C182F40401300E822788EC0FF0040101
:1041F0002C0E826F88EC0FF025C500F126C501F169
:1042000027C502F128C503F10101200E046F000E3D
:10421000056F000E066F000E076FB3EC3BF000C198
:1042200033F501C134F502C135F503C136F520EC93
:104230003CF02AC182F40401300E822788EC0FF092
:104240002BC182F40401300E822788EC0FF02CC1C0
:1042500082F40401300E822788EC0FF02DC182F425
:104260000401300E822788EC0FF02EC182F4040185
:10427000300E822788EC0FF02FC182F40401300E3B
:10428000822788EC0FF030C182F40401300E8227BF
:1042900088EC0FF031C182F40401300E822788ECE3
:1042A0000FF032C182F40401300E822788EC0FF047
:1042B00033C182F40401300E822788EC0FF092ECB7
:1042C0000FF0050133676CEF21F034676CEF21F0DC
:1042D00035676CEF21F0366702D00BEF22F0129EAB
:1042E000129C21C500F122C501F123C502F124C5AC
:1042F00003F1899A400EC76E200EC66E9E96C69E2A
:104300000B0EC96EFF0E9EB602D0E82EFCD79E960D
:10431000C69E02C1C9FFFF0E9EB602D0E82EFCD792
:104320009E96C69E01C1C9FFFF0E9EB602D0E82E22
:10433000FCD79E96C69E00C1C9FFFF0E9EB602D056
:10434000E82EFCD79E96C69EC952FF0E9EB602D09E
:10435000E82EFCD70501200E326F040114EE00F0A8
:1043600080517F0BE1269E96C69EC952FF0E9EB6D7
:1043700002D0E82EFCD7C9CFE7FF0401802B05014E
:10438000322FADEF21F0898A33C500F134C501F138
:1043900035C502F136C503F10101010E046F000EAF
:1043A000056F000E066F000E076F82EC3BF000C138
:1043B00033F501C134F502C135F503C136F5050108
:1043C0003367EAEF21F03467EAEF21F03567EAEF6F
:1043D00021F0366702D00BEF22F021C500F122C593
:1043E00001F123C502F124C503F10101200E046F80
:1043F000000E056F000E066F000E076F87EC3BF096
:1044000000C121F501C122F502C123F503C124F544
:10441000128EADEF34F00401450E826F88EC0FF080
:1044200004014F0E826F88EC0FF00401460E826F7C
:1044300088EC0FF038EF28F0078431EC47F097EC68
:104440003CF02DC500F120EC3CF004014C0E826FD5
:1044500088EC0FF00401300E826F88EC0FF004013D
:104460002C0E826F88EC0FF031C182F40401300E03
:10447000822788EC0FF032C182F40401300E8227CB
:1044800088EC0FF033C182F40401300E822788ECEF
:104490000FF004012C0E826F88EC0FF097EC3CF0CB
:1044A0002EC500F120EC3CF031C182F40401300E45
:1044B000822788EC0FF032C182F40401300E82278B
:1044C00088EC0FF033C182F40401300E822788ECAF
:1044D0000FF0079438EF28F004014C0E826F88EC3F
:1044E0000FF00401650E826F88EC0FF0D5EC40F000
:1044F00038EF28F004014C0E826F88EC0FF00401B5
:10450000450E826F88EC0FF0ECEC40F038EF28F0AD
:1045100004014C0E826F88EC0FF00401620E826F72
:1045200088EC0FF01AEC41F038EF28F004014C0E43
:10453000826F88EC0FF00401420E826F88EC0FF05E
:1045400003EC41F038EF28F004014C0E826F88EC48
:104550000FF00401760E826F88EC0FF004012C0E30
:10456000826F88EC0FF000012650FE0AD8B4C6EF27
:1045700022F000012650FD0AD8B4CDEF22F004014C
:10458000300E826F88EC0FF038EF28F00401310E06
:10459000826F88EC0FF038EF28F00401320E826F42
:1045A00088EC0FF038EF28F004014C0E826F88EC95
:1045B0000FF004015A0E826F88EC0FF004012C0EEC
:1045C000826F88EC0FF031EC47F097EC3CF005017E
:1045D0002E51130A06E005012E51170A0DE005EFD2
:1045E00023F00101000E006F000E016F100E026F2C
:1045F000000E036F05EF23F00101000E006F000EA7
:10460000016F000E026F010E036F0101200E046F97
:10461000000E056F000E066F000E076FB3EC3BF047
:1046200020EC3CF02AC182F40401300E822788EC91
:104630000FF02BC182F40401300E822788EC0FF0BA
:104640002CC182F40401300E822788EC0FF02DC1BA
:1046500082F40401300E822788EC0FF02EC182F420
:104660000401300E822788EC0FF02FC182F4040180
:10467000300E822788EC0FF030C182F40401300E36
:10468000822788EC0FF031C182F40401300E8227BA
:1046900088EC0FF032C182F40401300E822788ECDE
:1046A0000FF033C182F40401300E822788EC0FF042
:1046B00038EF28F0078404014C0E826F88EC0FF06D
:1046C0000401310E826F88EC0FF004012C0E826F12
:1046D00088EC0FF025C500F126C501F127C502F1D0
:1046E00028C503F10101200E046F000E056F000EB6
:1046F000066F000E076FB3EC3BF020EC3CF02AC1D4
:1047000082F40401300E822788EC0FF02BC182F472
:104710000401300E822788EC0FF02CC182F40401D2
:10472000300E822788EC0FF02DC182F40401300E88
:10473000822788EC0FF02EC182F40401300E82270C
:1047400088EC0FF02FC182F40401300E822788EC30
:104750000FF030C182F40401300E822788EC0FF094
:1047600031C182F40401300E822788EC0FF032C18F
:1047700082F40401300E822788EC0FF033C182F4FA
:104780000401300E822788EC0FF0079438EF28F0F0
:10479000078404014C0E826F88EC0FF00401320E86
:1047A000826F88EC0FF009EC43F0079438EF28F0A3
:1047B000078439B0DEEF23F0F1EF23F0010E176E1E
:1047C00004014C0E826F88EC0FF00401330E826FEF
:1047D00088EC0FF066EC43F0000E176E079465EF5F
:1047E00023F0020E176E66EC43F08B800501010E7C
:1047F000306F3C0E316F01015E6B5F6B606B616B04
:10480000626B636B646B656B666B676B686B696B24
:10481000536B546BCF6ACE6A0F9A0F9C0F9E030E98
:10482000176E04014C0E826F88EC0FF00401330EFA
:10483000826F88EC0FF004012C0E826F88EC0FF071
:1048400004012D0E826F88EC0FF00401310E826F8F
:1048500088EC0FF0ABEF34F066EC43F0000E176E0F
:104860008B90ADEF34F0078404014C0E826F88EC1E
:104870000FF00401340E826F88EC0FF004012C0E4F
:10488000826F88EC0FF0D8EC3CF084C32AF185C32A
:104890002BF186C32CF187C32DF188C32EF189C378
:1048A0002FF18AC330F18BC331F18CC332F18DC348
:1048B00033F10101296BE5EC3CF05CEC3CF0200E9F
:1048C000046F000E056F000E066F000E076F93EC6D
:1048D0003BF000C121F501C122F502C123F503C15E
:1048E00024F5E4EC46F038C5AFF539C5B0F53AC566
:1048F000B1F53BC5B2F53CC5B3F53DC5B4F53EC514
:10490000B5F5BCEC1EF004012C0E826F88EC0FF0A4
:104910003FC500F140C501F141C502F142C503F1B7
:104920000101000E046F000E056F010E066F000EF0
:10493000076FB3EC3BF020EC3CF02967A2EF24F0CA
:10494000A7EF24F004012D0E826F88EC0FF030C128
:1049500082F40401300E822788EC0FF031C182F41A
:104960000401300E822788EC0FF004012E0E826FB6
:1049700088EC0FF032C182F40401300E822788ECFB
:104980000FF033C182F40401300E822788EC0FF05F
:1049900004012C0E826F88EC0FF097EC3CF043C5BD
:1049A00000F144C501F1D7EC35F004012C0E826F03
:1049B00088EC0FF097EC3CF045C500F120EC3CF0A2
:1049C00031C182F40401300E822788EC0FF032C12D
:1049D00082F40401300E822788EC0FF033C182F498
:1049E0000401300E822788EC0FF004012C0E826F38
:1049F00088EC0FF00101036B026B4CC501F14BC554
:104A000000F101AF09EF25F00101FF0E026FFF0E6B
:104A1000036F20EC3CF0296710EF25F015EF25F02F
:104A200004012D0E826F88EC0FF02FC182F4040177
:104A3000300E822788EC0FF030C182F40401300E72
:104A4000822788EC0FF031C182F40401300E8227F6
:104A500088EC0FF032C182F40401300E822788EC1A
:104A60000FF033C182F40401300E822788EC0FF07E
:104A700004012C0E826F88EC0FF00101036B026BB6
:104A80004EC501F14DC500F101AF4CEF25F001011C
:104A9000FF0E026FFF0E036F20EC3CF0296753EF0F
:104AA00025F058EF25F004012D0E826F88EC0FF0F1
:104AB0002FC182F40401300E822788EC0FF030C140
:104AC00082F40401300E822788EC0FF031C182F4A9
:104AD0000401300E822788EC0FF032C182F4040109
:104AE000300E822788EC0FF033C182F40401300EBF
:104AF000822788EC0FF004012C0E826F88EC0FF0F7
:104B00000101036B026B50C501F14FC500F101AF0C
:104B10008FEF25F00101FF0E026FFF0E036F20ECF7
:104B20003CF0296796EF25F09BEF25F004012D0E50
:104B3000826F88EC0FF02FC182F40401300E8227BF
:104B400088EC0FF030C182F40401300E822788EC2B
:104B50000FF031C182F40401300E822788EC0FF08F
:104B600032C182F40401300E822788EC0FF033C189
:104B700082F40401300E822788EC0FF004012C0E21
:104B8000826F88EC0FF00101036B026B52C501F1DB
:104B900051C500F101AFD2EF25F00101FF0E026F08
:104BA000FF0E036F20EC3CF02967D9EF25F0DEEF14
:104BB00025F004012D0E826F88EC0FF02FC182F4D6
:104BC0000401300E822788EC0FF030C182F404011A
:104BD000300E822788EC0FF031C182F40401300ED0
:104BE000822788EC0FF032C182F40401300E822754
:104BF00088EC0FF033C182F40401300E822788EC78
:104C00000FF004012C0E826F88EC0FF00101036B92
:104C1000026B54C501F153C500F101AF15EF26F049
:104C20000101FF0E026FFF0E036F20EC3CF02967BD
:104C30001CEF26F021EF26F004012D0E826F88EC88
:104C40000FF02FC182F40401300E822788EC0FF0A0
:104C500030C182F40401300E822788EC0FF031C19C
:104C600082F40401300E822788EC0FF032C182F406
:104C70000401300E822788EC0FF033C182F4040166
:104C8000300E822788EC0FF004012C0E826F88EC26
:104C90000FF00101036B026B56C501F155C500F120
:104CA00001AF58EF26F00101FF0E026FFF0E036FF8
:104CB00020EC3CF029675FEF26F064EF26F004015A
:104CC0002D0E826F88EC0FF02FC182F40401300E9C
:104CD000822788EC0FF030C182F40401300E822765
:104CE00088EC0FF031C182F40401300E822788EC89
:104CF0000FF032C182F40401300E822788EC0FF0ED
:104D000033C182F40401300E822788EC0FF00401D5
:104D10002C0E826F88EC0FF00101036B026B4AC509
:104D200001F149C500F101AF9BEF26F00101FF0E33
:104D3000026FFF0E036F20EC3CF02967A2EF26F014
:104D4000A7EF26F004012D0E826F88EC0FF02FC123
:104D500082F40401300E822788EC0FF030C182F417
:104D60000401300E822788EC0FF031C182F4040177
:104D7000300E822788EC0FF032C182F40401300E2D
:104D8000822788EC0FF033C182F40401300E8227B1
:104D900088EC0FF004012C0E826F88EC0FF037C501
:104DA000E8FFE8B806D00401300E826F88EC0FF0FF
:104DB00005D00401310E826F88EC0FF0079438EFB4
:104DC00028F0D8EC3CF085C32AF186C32BF187C3C9
:104DD0002CF188C32DF189C32EF18AC32FF18BC327
:104DE00030F18CC331F18DC332F18EC333F1010147
:104DF000296BE5EC3CF05CEC3CF00101010E046F2A
:104E0000000E056F000E066F000E076F82EC3BF080
:104E1000100E046F000E056F000E066F000E076F78
:104E200093EC3BF000C129F501C12AF502C12BF535
:104E300003C12CF590EC42F004014C0E826F88EC1B
:104E40000FF00401460E826F88EC0FF004012C0E67
:104E5000826F88EC0FF025C500F126C501F127C54A
:104E600002F128C503F10101100E046F000E056F59
:104E7000000E066F000E076FB3EC3BF020EC3CF029
:104E80002AC182F40401300E822788EC0FF02BC176
:104E900082F40401300E822788EC0FF02CC182F4DA
:104EA0000401300E822788EC0FF02DC182F404013A
:104EB000300E822788EC0FF02EC182F40401300EF0
:104EC000822788EC0FF02FC182F40401300E822774
:104ED00088EC0FF030C182F40401300E822788EC98
:104EE0000FF031C182F40401300E822788EC0FF0FC
:104EF00032C182F40401300E822788EC0FF033C1F6
:104F000082F40401300E822788EC0FF038EF28F08D
:104F100039B08DEF27F0020E176E66EC43F00001FA
:104F20001750020AD8B4ABEF27F005012F51010A40
:104F3000D8B4A1EF27F015B2A6EF27F081BAA6EFFB
:104F400027F0000E176E1584ADEF34F0050E176EC6
:104F50001584D9EF47F08B8001015E6B5F6B606B4E
:104F6000616B626B636B646B656B666B676B686BC5
:104F7000696B536B546BCF6ACE6A0F9A0F9C0F9E6E
:104F8000030E176EADEF34F066EC43F005012F51C0
:104F9000010AD8B4D2EF27F015B2D7EF27F081BAC3
:104FA000D7EF27F0000E176E1584ADEF34F0050E25
:104FB000176E1584D9EF47F004014C0E826F88EC10
:104FC0000FF00401350E826F88EC0FF004012C0EF7
:104FD000826F88EC0FF097EC3CF00784B9C500F1C4
:104FE000079420EC3CF031C182F40401300E82279A
:104FF00088EC0FF032C182F40401300E822788EC75
:105000000FF033C182F40401300E822788EC0FF0D8
:1050100038EF28F029EC43F097EC3CF037C500F16D
:1050200020EC3CF004014C0E826F88EC0FF0040180
:10503000360E826F88EC0FF004012C0E826F88EC24
:105040000FF031C182F40401300E822788EC0FF09A
:1050500032C182F40401300E822788EC0FF033C194
:1050600082F40401300E822788EC0FF038EF28F02C
:1050700092EC0FF0ADEF34F004014C0E826F88EC2F
:105080000FF00401500E826F88EC0FF004012C0E1B
:10509000826F88EC0FF085C32AF186C32BF187C39A
:1050A0002CF188C32DF189C32EF18AC32FF18BC354
:1050B00030F18CC331F18DC332F18EC333F1010174
:1050C000E5EC3CF05CEC3CF003018451530A0DE04C
:1050D000030184514D0A38E00401780E826F88EC98
:1050E0000FF092EC0FF0ADEF34F00401530E826F2D
:1050F00088EC0FF0250E0C6E00C10BF0FBEC0BF0F2
:10510000260E0C6E01C10BF0FBEC0BF0270E0C6EA3
:1051100002C10BF0FBEC0BF0280E0C6E03C10BF080
:10512000FBEC0BF000C157F501C158F502C159F570
:1051300003C15AF500C15BF501C15CF502C15DF523
:1051400003C15EF519EF29F004014D0E826F88EC62
:105150000FF0290E0C6E00C10BF0FBEC0BF000C140
:105160005FF500C160F519EF29F004014C0E826F64
:1051700088EC0FF00401540E826F88EC0FF00401EC
:105180002C0E826F88EC0FF084C32AF185C32BF1BB
:1051900086C32CF187C32DF188C32EF189C32FF16B
:1051A0008AC330F18BC331F18DC332F18EC333F139
:1051B0000101E5EC3CF05CEC3CF00101000E046FF9
:1051C000000E056F010E066F000E076F93EC3BF0AB
:1051D000210E0C6E00C10BF0FBEC0BF0220E0C6EDE
:1051E00001C10BF0FBEC0BF0230E0C6E02C10BF0B7
:1051F000FBEC0BF0240E0C6E03C10BF0FBEC0BF080
:1052000000C161F501C162F502C163F503C164F536
:1052100019EF29F004014C0E826F88EC0FF00401A5
:10522000490E826F88EC0FF004012C0E826F88EC1F
:105230000FF0250E12EC0CF0E8CF00F1260E12EC68
:105240000CF0E8CF01F1270E12EC0CF0E8CF02F1E0
:10525000280E12EC0CF0E8CF03F120EC3CF0E3EC6C
:1052600039F00401730E826F88EC0FF004012C0EEC
:10527000826F88EC0FF097EC3CF0290E12EC0CF0EA
:10528000E8CF00F120EC3CF0E3EC39F004016D0EC6
:10529000826F88EC0FF004012C0E826F88EC0FF007
:1052A0005BC500F15CC501F15DC502F15EC503F1AE
:1052B00020EC3CF0E3EC39F00401730E826F88ECD3
:1052C0000FF004012C0E826F88EC0FF097EC3CF08D
:1052D00060C500F120EC3CF0E3EC39F004016D0E08
:1052E000826F88EC0FF004012C0E826F88EC0FF0B7
:1052F00061C500F162C501F163C502F164C503F146
:10530000C8EC34F004012C0E826F88EC0FF092ECA4
:105310000FF0ADEF34F083C32AF184C32BF185C3C2
:105320002CF186C32DF187C32EF188C32FF189C3D9
:1053300030F18AC331F18BC332F18CC333F10101F7
:10534000E5EC3CF05CEC3CF0160E0C6E00C10BF092
:10535000FBEC0BF0170E0C6E01C10BF0FBEC0BF02D
:10536000180E0C6E02C10BF0FBEC0BF0190E0C6E5C
:1053700003C10BF0FBEC0BF000C18EF101C18FF10A
:1053800002C190F103C191F100C192F101C193F109
:1053900002C194F103C195F16DEF2AF083C32AF1A4
:1053A00084C32BF185C32CF186C32DF187C32EF165
:1053B00088C32FF189C330F18AC331F18BC332F135
:1053C0008CC333F10101E5EC3CF05CEC3CF000C136
:1053D0008EF101C18FF102C190F103C191F100C1C1
:1053E00092F101C193F102C194F103C195F16DEF06
:1053F0002AF083C32AF184C32BF185C32CF186C321
:105400002DF187C32EF188C32FF189C330F18AC3F0
:1054100031F18CC332F18DC333F10101E5EC3CF085
:105420005CEC3CF00101000E046F000E056F010EF4
:10543000066F000E076F93EC3BF01A0E0C6E00C166
:105440000BF0FBEC0BF01B0E0C6E01C10BF0FBEC38
:105450000BF01C0E0C6E02C10BF0FBEC0BF01D0EE2
:105460000C6E03C10BF0FBEC0BF000C196F101C117
:1054700097F102C198F103C199F16DEF2AF083C34E
:105480002AF184C32BF185C32CF186C32DF187C388
:105490002EF188C32FF189C330F18AC331F18CC357
:1054A00032F18DC333F10101E5EC3CF05CEC3CF0F2
:1054B0000101000E046F000E056F010E066F000E55
:1054C000076F93EC3BF000C196F101C197F102C167
:1054D00098F103C199F16DEF2AF0160E12EC0CF061
:1054E000E8CF00F1170E12EC0CF0E8CF01F1180E26
:1054F00012EC0CF0E8CF02F1190E12EC0CF0E8CF30
:1055000003F120EC3CF0E3EC39F00401730E826F00
:1055100088EC0FF004012C0E826F88EC0FF08EC126
:1055200000F18FC101F190C102F191C103F120ECB2
:105530003CF0E3EC39F00401730E826F88EC0FF05D
:1055400004012C0E826F88EC0FF01A0E12EC0CF096
:10555000E8CF00F11B0E12EC0CF0E8CF01F11C0EAD
:1055600012EC0CF0E8CF02F11D0E12EC0CF0E8CFBB
:1055700003F1C8EC34F004012C0E826F88EC0FF0BC
:1055800096C100F197C101F198C102F199C103F1EF
:10559000C8EC34F092EC0FF0ADEF34F00401690E7A
:1055A000826F88EC0FF004012C0E826F88EC0FF0F4
:1055B0000101040E006F000E016F000E026F000E5D
:1055C000036F20EC3CF02CC182F40401300E8227E2
:1055D00088EC0FF02DC182F40401300E822788EC94
:1055E0000FF02EC182F40401300E822788EC0FF0F8
:1055F0002FC182F40401300E822788EC0FF030C1F5
:1056000082F40401300E822788EC0FF031C182F45D
:105610000401300E822788EC0FF032C182F40401BD
:10562000300E822788EC0FF033C182F40401300E73
:10563000822788EC0FF004012C0E826F88EC0FF0AB
:1056400001010B0E006F000E016F000E026F000EC5
:10565000036F20EC3CF02CC182F40401300E822751
:1056600088EC0FF02DC182F40401300E822788EC03
:105670000FF02EC182F40401300E822788EC0FF067
:105680002FC182F40401300E822788EC0FF030C164
:1056900082F40401300E822788EC0FF031C182F4CD
:1056A0000401300E822788EC0FF032C182F404012D
:1056B000300E822788EC0FF033C182F40401300EE3
:1056C000822788EC0FF004012C0E826F88EC0FF01B
:1056D0000101540E006F000E016F000E026F000EEC
:1056E000036F20EC3CF02CC182F40401300E8227C1
:1056F00088EC0FF02DC182F40401300E822788EC73
:105700000FF02EC182F40401300E822788EC0FF0D6
:105710002FC182F40401300E822788EC0FF030C1D3
:1057200082F40401300E822788EC0FF031C182F43C
:105730000401300E822788EC0FF032C182F404019C
:10574000300E822788EC0FF033C182F40401300E52
:10575000822788EC0FF004012C0E826F88EC0FF08A
:10576000200EF86EF76AF66A04010900F5CF82F49C
:1057700088EC0FF00900F5CF82F488EC0FF00900F7
:10578000F5CF82F488EC0FF00900F5CF82F488ECB5
:105790000FF00900F5CF82F488EC0FF00900F5CF87
:1057A00082F488EC0FF00900F5CF82F488EC0FF05A
:1057B0000900F5CF82F488EC0FF092EC0FF0ADEF1A
:1057C00034F08351630AD8A4ABEF34F08451610AFA
:1057D000D8A4ABEF34F085516C0AD8A4ABEF34F009
:1057E0008651410A3FE08651440A1BE08651420A35
:1057F000D8B445EF2CF08651350AD8B437EF36F0DF
:105800008651360AD8B48CEF36F08651370AD8B4B0
:10581000F5EF36F08651380AD8B453EF37F0ABEFD6
:1058200034F00798079A04017A0E826F88EC0FF023
:105830000401780E826F88EC0FF00401640E826F11
:1058400088EC0FF00401550E826F88EC0FF02EEFFC
:105850002CF004014C0E826F88EC0FF092EC0FF0EC
:10586000ADEF34F00788079A04017A0E826F88EC56
:105870000FF00401410E826F88EC0FF00401610EFD
:10588000826F88EC0FF022EF2CF00798078A040152
:105890007A0E826F88EC0FF00401420E826F88EC62
:1058A0000FF00401610E826F88EC0FF022EF2CF0F4
:1058B0000101666763EF2CF0676763EF2CF06867A0
:1058C00063EF2CF0696716D001014F676FEF2CF082
:1058D00050676FEF2CF051676FEF2CF052670AD0D2
:1058E0000101000E006F000E016F000E026F000E2E
:1058F000036F120011B80AD00101620E046F010E8D
:10590000056F000E066F000E076F09D00101A70E8C
:10591000046F020E056F000E066F000E076F66C162
:1059200000F167C101F168C102F169C103F182ECC4
:105930003BF003BF0CEF2DF0119A119C0101000EFA
:10594000046FA80E056F550E066F020E076F66C135
:1059500000F167C101F168C102F169C103F166C1DB
:105960008AF167C18BF168C18CF169C18DF182EC5C
:105970003BF003BF0BD00101000E8A6FA80E8B6FA6
:10598000550E8C6F020E8D6F118A119C0E0E12EC4B
:105990000CF0E8CF18F10F0E12EC0CF0E8CF19F173
:1059A000100E12EC0CF0E8CF1AF1110E12EC0CF004
:1059B000E8CF1BF1CBEC3AF08AC104F18BC105F1C1
:1059C0008CC106F18DC107F182EC3BF007828FECB0
:1059D0003AF0CBEC3AF007928FEC3AF08AC100F142
:1059E0008BC101F18CC102F18DC103F107928FECE3
:1059F0003AF0CC0E046FE00E056F870E066F050EB1
:105A0000076F82EC3BF000C118F101C119F102C12E
:105A10001AF103C11BF140D013AA11EF2DF0138E20
:105A2000139A119C119A0101800E006F1A0E016FDA
:105A3000060E026F000E036F4FC104F150C105F155
:105A400051C106F152C107F182EC3BF003AF05D022
:105A500097EC3CF0118C119A12000E0E12EC0CF027
:105A6000E8CF18F10F0E12EC0CF0E8CF19F1100E80
:105A700012EC0CF0E8CF1AF1110E12EC0CF0E8CF9A
:105A80001BF14FC100F150C101F151C102F152C1EE
:105A900003F107828FEC3AF018C100F119C101F14E
:105AA0001AC102F11BC103F112000784BAC166F1E9
:105AB000BBC167F1BCC168F1BDC169F14BC14FF118
:105AC0004CC150F14DC151F14EC152F157C159F184
:105AD00058C15AF107940101666776EF2DF06767A8
:105AE00076EF2DF0686776EF2DF0696716D001012B
:105AF0004F6782EF2DF0506782EF2DF0516782EFF4
:105B00002DF052670AD00101000E006F000E016FE8
:105B1000000E026F000E036F120011B80AD00101CF
:105B2000620E046F010E056F000E066F000E076F08
:105B300009D00101A70E046F020E056F000E066F5B
:105B4000000E076F66C100F167C101F168C102F183
:105B500069C103F182EC3BF003BF0EEF2EF00101AF
:105B6000000E046FA80E056F550E066F020E076F2C
:105B700066C100F167C101F168C102F169C103F1B9
:105B800066C18AF167C18BF168C18CF169C18DF181
:105B900082EC3BF003BF09D00101000E8A6FA80E12
:105BA0008B6F550E8C6F020E8D6FCBEC3AF000C1EF
:105BB00004F101C105F102C106F103C107F1000EB4
:105BC000006FA00E016F980E026F7B0E036FB3EC97
:105BD0003BF000C118F101C119F102C11AF103C172
:105BE0001BF1000E006FA00E016F980E026F7B0E6E
:105BF000036F8AC104F18BC105F18CC106F18DC11F
:105C000007F1B3EC3BF018C104F119C105F11AC159
:105C100006F11BC107F182EC3BF012000101A80E56
:105C2000006F610E016F000E026F000E036F4FC117
:105C300004F150C105F151C106F152C107F182ECE6
:105C40003BF003AF0AD00101A80E006F610E016F97
:105C5000000E026F000E036F00D0C80E006FAF0E73
:105C6000016F000E026F000E036F4FC104F150C1AF
:105C700005F151C106F152C107F193EC3BF012005E
:105C80000784BAC166F1BBC167F1BCC168F1BDC18F
:105C900069F14BC14FF14CC150F14DC151F14EC1B1
:105CA00052F157C159F158C15AF107940101666781
:105CB00061EF2EF0676761EF2EF0686761EF2EF0FD
:105CC000696716D001014F676DEF2EF050676DEFD9
:105CD0002EF051676DEF2EF052670AD00101000ED1
:105CE000006F000E016F000E026F000E036F1200B6
:105CF00011B80AD00101620E046F010E056F000E8B
:105D0000066F000E076F09D00101A70E046F020E87
:105D1000056F000E066F000E076F66C100F167C1C8
:105D200001F168C102F169C103F182EC3BF003BFEC
:105D300023EF2FF00101000E046FA80E056F550E22
:105D4000066F020E076F66C100F167C101F168C1FD
:105D500002F169C103F166C18AF167C18BF168C1C3
:105D60008CF169C18DF182EC3BF003BF09D00101D8
:105D7000000E8A6FA80E8B6F550E8C6F020E8D6F02
:105D8000010E006F000E016F000E026F000E036F18
:105D90008AC104F18BC105F18CC106F18DC107F1F7
:105DA000B3EC3BF018C104F119C105F11AC106F1B9
:105DB0001BC107F120EC3CF02AC182F40401300E33
:105DC000822788EC0FF02BC182F40401300E822769
:105DD00088EC0FF02CC182F40401300E822788EC8D
:105DE0000FF02DC182F40401300E822788EC0FF0F1
:105DF0002EC182F40401300E822788EC0FF02FC1EF
:105E000082F40401300E822788EC0FF030C182F456
:105E10000401300E822788EC0FF031C182F40401B6
:105E2000300E822788EC0FF032C182F40401300E6C
:105E3000822788EC0FF033C182F40401300E8227F0
:105E400088EC0FF012004FC100F150C101F151C1B7
:105E500002F152C103F1010120EC3CF0E3EC39F016
:105E600012000401730E826F88EC0FF004012C0EF7
:105E7000826F88EC0FF0078462C166F163C167F13D
:105E800064C168F165C169F14BC14FF14CC150F17A
:105E90004DC151F14EC152F157C159F158C15AF19A
:105EA000079457EC2FF092EC0FF0ADEF34F066C191
:105EB00000F167C101F168C102F169C103F101019B
:105EC00020EC3CF0E3EC39F00401630E826F88ECC7
:105ED0000FF004012C0E826F88EC0FF04FC100F11F
:105EE00050C101F151C102F152C103F1010120EC95
:105EF0003CF0E3EC39F00401660E826F88EC0FF0A1
:105F000004012C0E826F88EC0FF097EC3CF059C125
:105F100000F15AC101F1010120EC3CF0E3EC39F051
:105F20000401740E826F88EC0FF0120010820401DD
:105F3000530E826F88EC0FF004012C0E826F88ECF8
:105F40000FF083C32AF184C32BF185C32CF186C3E0
:105F50002DF187C32EF188C32FF189C330F18AC395
:105F600031F18BC332F18CC333F10101E5EC3CF02C
:105F70005CEC3CF000C166F101C167F102C168F15F
:105F800003C169F18EC32AF18FC32BF190C32CF1A9
:105F900091C32DF192C32EF193C32FF194C330F12D
:105FA00095C331F196C332F197C333F10101E5ECAA
:105FB0003CF05CEC3CF000C14FF101C150F102C17A
:105FC00051F103C152F1D8EC3CF099C32FF19AC3BF
:105FD00030F19BC331F19CC332F19DC333F1010118
:105FE000E5EC3CF05CEC3CF000C159F101C15AF128
:105FF00057EC2FF004012C0E826F88EC0FF011EF9C
:1060000030F0118E1DA002D01DAE108C1CBE02D02F
:106010001CA4108E03018251520A02E10F8201D0AA
:106020000F928251750A02E1108401D010948251BE
:10603000550A02E1108601D010968351310A03E11E
:106040001382138402D01392139403018351660ABE
:1060500001E056D00401660E826F88EC0FF0040157
:106060002C0E826F88EC0FF055EC2DF020EC3CF0FC
:106070002AC182F40401300E822788EC0FF02BC174
:1060800082F40401300E822788EC0FF02CC182F4D8
:106090000401300E822788EC0FF02DC182F4040138
:1060A000300E822788EC0FF02EC182F40401300EEE
:1060B000822788EC0FF02FC182F40401300E822772
:1060C00088EC0FF030C182F40401300E822788EC96
:1060D0000FF031C182F40401300E822788EC0FF0FA
:1060E00032C182F40401300E822788EC0FF033C1F4
:1060F00082F40401300E822788EC0FF0ABEF34F00D
:1061000011A003D011A401D01084078410B2EAEFCB
:1061100030F010A4CEEF30F0BAC166F1BBC167F128
:10612000BCC168F1BDC169F1BEC16AF1BFC16BF10B
:10613000C0C16CF1C1C16DF1C2C16EF1C3C16FF1DB
:10614000C4C170F1C5C171F1C6C172F1C7C173F1AB
:10615000C8C174F1C9C175F1CAC176F1CBC177F17B
:10616000CCC178F1CDC179F1CEC17AF1CFC17BF14B
:10617000D0C17CF1D1C17DF1D2C17EF1D3C17FF11B
:10618000D4C180F1D5C181F1D6C182F1D7C183F1EB
:10619000D8C184F1D9C185F1D6EF30F062C166F182
:1061A00063C167F164C168F165C169F1BAC186F183
:1061B000BBC187F1BCC188F1BDC189F14BC14FF1B1
:1061C0004CC150F14DC151F14EC152F157C159F17D
:1061D00058C15AF107940FA00CEF31F001019667F6
:1061E000F9EF30F09767F9EF30F09867F9EF30F09A
:1061F0009967FDEF30F00CEF31F058EC2CF096C1C0
:1062000004F197C105F198C106F199C107F182EC3B
:106210003BF003BF71EF34F058EC2CF00101000E9D
:10622000046F000E056F010E066F000E076FB3ECD2
:106230003BF011A02AD011A228D020EC3CF0296715
:1062400001D005D004012D0E826F88EC0FF030C113
:1062500082F40401300E822788EC0FF031C182F401
:106260000401300E822788EC0FF032C182F4040161
:10627000300E822788EC0FF033C182F40401300E17
:10628000822788EC0FF092EC0FF012A8C5D012987C
:106290001EC01FF01F3A1F42070E1F1600011F509D
:1062A000000AD8B4D8EF31F000011F50010AD8B469
:1062B00064EF31F000011F50020AD8B462EF31F0F0
:1062C0000AEF32F00AEF32F097EC3CF02FC001F108
:1062D00030C000F1D89001330033D890013300333F
:1062E0000101630E046F000E056F000E066F000EB5
:1062F000076FB3EC3BF0280E046F000E056F000E25
:10630000066F000E076F82EC3BF000C132F097EC95
:106310003CF02DC001F1019F019D2EC000F1010153
:10632000A40E046F000E056F000E066F000E076FBF
:10633000B3EC3BF000C131F000C104F101C105F143
:1063400002C106F103C107F1640E006F000E016F78
:10635000000E026F000E036F82EC3BF0050E046F1F
:10636000000E056F000E066F000E076FB3EC3BF0DA
:1063700000C104F101C105F102C106F103C107F139
:1063800097EC3CF032C000F182EC3BF000C133F0FE
:1063900033C0E8FF050F325C03E78A840AEF32F06E
:1063A00033C0E8FF0A0F325C01E68A940AEF32F04C
:1063B00000C124F101C125F102C126F103C127F179
:1063C00097EC3CF09DEC3CF01E501F0BE8CF00F129
:1063D0000101640E046F000E056F000E066F000EC3
:1063E000076F93EC3BF024C104F125C105F126C1F0
:1063F00006F127C107F182EC3BF003BF02D08A947B
:1064000001D08A8424C100F125C101F126C102F125
:1064100027C103F1ADEF34F000C124F101C125F132
:1064200002C126F103C127F110AE4DD0109E00C16C
:1064300008F101C109F102C10AF103C10BF120EC1D
:106440003CF030C1E2F131C1E3F132C1E4F133C1DA
:10645000E5F108C100F109C101F10AC102F10BC166
:1064600003F101016C0E046F070E056F000E066F3D
:10647000000E076F82EC3BF003BF04D00101550E04
:10648000E66F1CD008C100F109C101F10AC102F197
:106490000BC103F10101A40E046F060E056F000E7F
:1064A000066F000E076F82EC3BF003BF04D00101C2
:1064B0007F0EE66F03D00101FF0EE66F208E11AE56
:1064C00071EF34F0119E24C100F125C101F126C104
:1064D00002F127C103F111A005D011A203D00FB022
:1064E00071EF34F010A47CEF32F00401750E826F6E
:1064F00088EC0FF081EF32F00401720E826F88ECAD
:106500000FF004012C0E826F88EC0FF020EC3CF0B1
:10651000296790EF32F00401200E826F93EF32F082
:1065200004012D0E826F88EC0FF030C182F404015B
:10653000300E822788EC0FF031C182F40401300E56
:10654000822788EC0FF004012E0E826F88EC0FF08A
:1065500032C182F40401300E822788EC0FF033C17F
:1065600082F40401300E822788EC0FF004016D0ED6
:10657000826F88EC0FF004012C0E826F88EC0FF014
:106580004FC100F150C101F151C102F152C103F1FB
:10659000010120EC3CF0E3EC39F00401480E826F7D
:1065A00088EC0FF004017A0E826F88EC0FF0040182
:1065B0002C0E826F88EC0FF066C100F167C101F10B
:1065C00068C102F169C103F1010120EC3CF0E3EC88
:1065D00039F00401630E826F88EC0FF004012C0E79
:1065E000826F88EC0FF066C100F167C101F168C1EC
:1065F00002F169C103F101010A0E046F000E056F7B
:10660000000E066F000E076F93EC3BF0000E046F58
:10661000120E056F000E066F000E076FB3EC3BF015
:1066200020EC3CF02AC182F40401300E822788EC71
:106630000FF02BC182F40401300E822788EC0FF09A
:106640002CC182F40401300E822788EC0FF02DC19A
:1066500082F40401300E822788EC0FF02EC182F400
:106660000401300E822788EC0FF02FC182F4040160
:10667000300E822788EC0FF030C182F40401300E16
:10668000822788EC0FF004012E0E826F88EC0FF049
:1066900031C182F40401300E822788EC0FF032C140
:1066A00082F40401300E822788EC0FF033C182F4AB
:1066B0000401300E822788EC0FF00401730E826F04
:1066C00088EC0FF004012C0E826F88EC0FF097EC31
:1066D0003CF059C100F15AC101F1D7EC35F003018A
:1066E0008351320A01E027D004012C0E826F88EC1E
:1066F0000FF097EC3CF00784B9C500F1079420EC4B
:106700003CF031C182F40401300E822788EC0FF096
:1067100032C182F40401300E822788EC0FF033C1BD
:1067200082F40401300E822788EC0FF00401420E3F
:10673000826F88EC0FF013A2EDEF33F004012C0E02
:10674000826F88EC0FF086C166F187C167F188C15E
:1067500068F189C169F158EC2CF00101000E046F59
:10676000000E056F010E066F000E076FB3EC3BF0D5
:1067700020EC3CF02967C2EF33F00401200E826F59
:10678000C5EF33F004012D0E826F88EC0FF030C19D
:1067900082F40401300E822788EC0FF031C182F4BC
:1067A0000401300E822788EC0FF004012E0E826F58
:1067B00088EC0FF032C182F40401300E822788EC9D
:1067C0000FF033C182F40401300E822788EC0FF001
:1067D00004016D0E826F88EC0FF003018351460AAD
:1067E00001E007D004012C0E826F88EC0FF040EC22
:1067F0002EF013A420EF34F004012C0E826F88ECED
:106800000FF013AC0EEF34F00401500E826F88ECE1
:106810000FF0139C1398139A20EF34F013AE1BEF74
:1068200034F00401460E826F88EC0FF0139E13982B
:10683000139A20EF34F00401530E826F88EC0FF0AE
:1068400039B037EF34F004012C0E826F88EC0FF072
:106850008BB032EF34F00401440E826F88EC0FF0FD
:1068600037EF34F00401530E826F88EC0FF00FB253
:106870003DEF34F00FA06FEF34F004012C0E826F67
:1068800088EC0FF0200EF86EF76AF66A0401090032
:10689000F5CF82F488EC0FF00900F5CF82F488EC94
:1068A0000FF00900F5CF82F488EC0FF00900F5CF66
:1068B00082F488EC0FF00900F5CF82F488EC0FF039
:1068C0000900F5CF82F488EC0FF00900F5CF82F4CF
:1068D00088EC0FF00900F5CF82F488EC0FF092EC11
:1068E0000FF00F90109E1298ADEF34F00401630E7C
:1068F000826F88EC0FF004012C0E826F88EC0FF091
:10690000B3EC34F004012C0E826F88EC0FF026EC0F
:1069100035F004012C0E826F88EC0FF0A2EC35F0FC
:1069200004012C0E826F88EC0FF00101F80E006F4D
:10693000CD0E016F660E026F030E036FC8EC34F0CC
:1069400004012C0E826F88EC0FF0B8EC35F092EC5D
:106950000FF0ADEF34F092EC0FF00301C26B079033
:106960001092BCEF37F0D8900E0E12EC0CF0E8CF7E
:1069700000F10F0E12EC0CF0E8CF01F1100E12EC4A
:106980000CF0E8CF02F1110E12EC0CF0E8CF03F19D
:106990000101000E046F000E056F010E066F000E60
:1069A000076FB3EC3BF020EC3CF02AC182F4040109
:1069B000300E822788EC0FF02BC182F40401300ED8
:1069C000822788EC0FF02CC182F40401300E82275C
:1069D00088EC0FF02DC182F40401300E822788EC80
:1069E0000FF02EC182F40401300E822788EC0FF0E4
:1069F0002FC182F40401300E822788EC0FF030C1E1
:106A000082F40401300E822788EC0FF031C182F449
:106A10000401300E822788EC0FF004012E0E826FE5
:106A200088EC0FF032C182F40401300E822788EC2A
:106A30000FF033C182F40401300E822788EC0FF08E
:106A400004016D0E826F88EC0FF01200120E12EC32
:106A50000CF0E8CF00F1130E12EC0CF0E8CF01F1CE
:106A6000140E12EC0CF0E8CF02F1150E12EC0CF043
:106A7000E8CF03F101010A0E046F000E056F000E4E
:106A8000066F000E076F93EC3BF0000E046F120EC2
:106A9000056F000E066F000E076FB3EC3BF020ECA5
:106AA0003CF02AC182F40401300E822788EC0FF0FA
:106AB0002BC182F40401300E822788EC0FF02CC128
:106AC00082F40401300E822788EC0FF02DC182F48D
:106AD0000401300E822788EC0FF02EC182F40401ED
:106AE000300E822788EC0FF02FC182F40401300EA3
:106AF000822788EC0FF030C182F40401300E822727
:106B000088EC0FF004012E0E826F88EC0FF031C17B
:106B100082F40401300E822788EC0FF032C182F437
:106B20000401300E822788EC0FF033C182F4040197
:106B3000300E822788EC0FF00401730E826F88EC10
:106B40000FF012000A0E12EC0CF0E8CF00F10B0E61
:106B500012EC0CF0E8CF01F10C0E12EC0CF0E8CFC7
:106B600002F10D0E12EC0CF0E8CF03F1D7EF35F087
:106B7000060E12EC0CF0E8CF00F1070E12EC0CF050
:106B8000E8CF01F1080E12EC0CF0E8CF02F1090E8B
:106B900012EC0CF0E8CF03F1D7EF35F0010197ECE0
:106BA0003CF0078457C100F158C101F1079401017D
:106BB000E80E046F800E056F000E066F000E076F63
:106BC00093EC3BF0000E046F040E056F000E066F91
:106BD000000E076FB3EC3BF0880E046F130E056FC9
:106BE000000E066F000E076F82EC3BF00A0E046F7A
:106BF000000E056F000E066F000E076FB3EC3BF042
:106C000020EC3CF0010129670BEF36F00401200E67
:106C1000826F0EEF36F004012D0E826F88EC0FF0BC
:106C200030C182F40401300E822788EC0FF031C1AC
:106C300082F40401300E822788EC0FF032C182F416
:106C40000401300E822788EC0FF004012E0E826FB3
:106C500088EC0FF033C182F40401300E822788ECF7
:106C60000FF00401430E826F88EC0FF0120087C30F
:106C70002AF188C32BF189C32CF18AC32DF18BC370
:106C80002EF18CC32FF18DC330F18EC331F190C33F
:106C900032F191C333F10101296BE5EC3CF05CEC7E
:106CA0003CF00101000E046F000E056F010E066F2F
:106CB000000E076F93EC3BF00E0E0C6E00C10BF054
:106CC000FBEC0BF00F0E0C6E01C10BF0FBEC0BF0AC
:106CD000100E0C6E02C10BF0FBEC0BF0110E0C6EE3
:106CE00003C10BF0FBEC0BF004017A0E826F88EC11
:106CF0000FF004012C0E826F88EC0FF00401350EAA
:106D0000826F88EC0FF004012C0E826F88EC0FF07C
:106D1000B3EC34F02EEF2CF087C32AF188C32BF1AB
:106D200089C32CF18AC32DF18BC32EF18CC32FF1B3
:106D30008DC330F18EC331F190C332F191C333F181
:106D40000101296BE5EC3CF05CEC3CF0880E046F33
:106D5000130E056F000E066F000E076F87EC3BF0F9
:106D6000000E046F040E056F000E066F000E076F15
:106D700093EC3BF00101E80E046F800E056F000EEE
:106D8000066F000E076FB3EC3BF00A0E0C6E00C1ED
:106D90000BF0FBEC0BF00B0E0C6E01C10BF0FBECDF
:106DA0000BF00C0E0C6E02C10BF0FBEC0BF00D0E99
:106DB0000C6E03C10BF0FBEC0BF004017A0E826F3A
:106DC00088EC0FF004012C0E826F88EC0FF00401A8
:106DD000360E826F88EC0FF004012C0E826F88EC67
:106DE0000FF0A2EC35F02EEF2CF087C32AF188C308
:106DF0002BF189C32CF18AC32DF18BC32EF18CC3E7
:106E00002FF18DC330F18FC331F190C332F191C3B3
:106E100033F10101E5EC3CF05CEC3CF0000E046F5A
:106E2000120E056F000E066F000E076F93EC3BF01D
:106E300001010A0E046F000E056F000E066F000EB2
:106E4000076FB3EC3BF0120E0C6E00C10BF0FBECC5
:106E50000BF0130E0C6E01C10BF0FBEC0BF0140EDB
:106E60000C6E02C10BF0FBEC0BF0150E0C6E03C1A7
:106E70000BF0FBEC0BF004017A0E826F88EC0FF044
:106E800004012C0E826F88EC0FF00401370E826F24
:106E900088EC0FF004012C0E826F88EC0FF026ECCA
:106EA00035F02EEF2CF087C32AF188C32BF189C36C
:106EB0002CF18AC32DF18BC32EF18CC32FF18DC31E
:106EC00030F18EC331F190C332F191C333F101013E
:106ED000296BE5EC3CF05CEC3CF0880E046F130E83
:106EE000056F000E066F000E076F87EC3BF0000E7B
:106EF000046F040E056F000E066F000E076F93EC13
:106F00003BF00101E80E046F800E056F000E066F66
:106F1000000E076FB3EC3BF0060E0C6E00C10BF0D9
:106F2000FBEC0BF0070E0C6E01C10BF0FBEC0BF051
:106F3000080E0C6E02C10BF0FBEC0BF0090E0C6E90
:106F400003C10BF0FBEC0BF004017A0E826F88ECAE
:106F50000FF004012C0E826F88EC0FF00401380E44
:106F6000826F88EC0FF004012C0E826F88EC0FF01A
:106F7000B8EC35F02EEF2CF007A82FEF38F0010118
:106F8000800E006F1A0E016F060E026F000E036F67
:106F90004BC104F14CC105F14DC106F14EC107F1E1
:106FA00082EC3BF003BF75EF38F0DDEC39F04BC1FC
:106FB00000F14CC101F14DC102F14EC103F1078254
:106FC0008FEC3AF018C104F119C105F11AC106F1AC
:106FD0001BC107F1F80E006FCD0E016F660E026F38
:106FE000030E036F82EC3BF00E0E0C6E00C10BF033
:106FF000FBEC0BF00F0E0C6E01C10BF0FBEC0BF079
:10700000100E0C6E02C10BF0FBEC0BF0110E0C6EAF
:1070100003C10BF0FBEC0BF00784010197EC3CF093
:1070200057C100F158C101F107940A0E0C6E00C15E
:107030000BF0FBEC0BF00B0E0C6E01C10BF0FBEC3C
:107040000BF00C0E0C6E02C10BF0FBEC0BF00D0EF6
:107050000C6E03C10BF0FBEC0BF075EF38F007AAD8
:1070600075EF38F00784010197EC3CF057C100F14F
:1070700058C101F10794060E0C6E00C10BF0FBEC39
:107080000BF0070E0C6E01C10BF0FBEC0BF0080EC1
:107090000C6E02C10BF0FBEC0BF0090E0C6E03C181
:1070A0000BF0FBEC0BF0078462C100F163C101F14E
:1070B00064C102F165C103F10794120E0C6E00C1A8
:1070C0000BF0FBEC0BF0130E0C6E01C10BF0FBECA4
:1070D0000BF0140E0C6E02C10BF0FBEC0BF0150E56
:1070E0000C6E03C10BF0FBEC0BF00798079A040140
:1070F000805181197F0B0DE09EA8FED714EE00F0A1
:1071000081517F0BE126E750812B0F01AD6E77EFA8
:1071100038F005012F51000AD8B4B8EF38F081BA21
:107120009DEF38F015B2B8EF38F005012F51010A84
:10713000D8B4B6EF38F0AFEF38F005012F51000AA0
:10714000D8B4D9EF47F005012F51010AD8B4B6EFF2
:1071500038F000011750050AD8B4D9EF47F081B8CC
:10716000B8EF38F05FEC3FF005EC40F070EC47F022
:10717000B1EF0EF006013251385D3351D8A0010F46
:10718000395D800BD8A4C9EF38F032C638F633C663
:1071900039F6120006013251365D3351D8A0010F85
:1071A000375D800BD8B4D9EF38F032C636F633C627
:1071B00037F6120007841AC632F61BC633F61CC611
:1071C00038F61DC639F6BAEC38F01EC632F61FC6C0
:1071D00033F6BAEC38F020C632F621C633F6BAECF4
:1071E00038F01AC632F61BC633F61CC636F61DC674
:1071F00037F6CAEC38F01EC632F61FC633F6CAECB4
:1072000038F020C632F621C633F6CAEC38F03851D1
:10721000365F3951D8A03929375F97EC3CF036C634
:1072200000F137C601F1A3EC3CF000C13AF601C110
:107230003BF622C632F623C633F624C638F625C6F8
:1072400039F6BAEC38F026C632F627C633F6BAEC71
:1072500038F028C632F629C633F6BAEC38F022C622
:1072600032F623C633F624C636F625C637F6CAEC00
:1072700038F026C632F627C633F6CAEC38F028C6F0
:1072800032F629C633F6CAEC38F03851365F395138
:10729000D8A03929375F97EC3CF036C600F137C6E5
:1072A00001F1A3EC3CF000C13CF601C13DF62AC659
:1072B00032F62BC633F62CC638F62DC639F6BAECA4
:1072C00038F02EC632F62FC633F6BAEC38F030C698
:1072D00032F631C633F6BAEC38F02AC632F62BC68F
:1072E00033F62CC636F62DC637F6CAEC38F02EC665
:1072F00032F62FC633F6CAEC38F030C632F631C655
:1073000033F6CAEC38F03851365F3951D8A03929F4
:10731000375F97EC3CF036C600F137C601F1A3ECBD
:107320003CF000C13EF601C13FF63AC632F63BC61C
:1073300033F63CC636F63DC637F6CAEC38F03EC6E4
:1073400032F63FC633F6CAEC38F00794120018C183
:1073500000F119C101F11AC102F11BC103F1000EC4
:10736000046F000E056F010E066F000E076FB3EC81
:107370003BF029A1D2EF39F02051D8B4D2EF39F047
:1073800018C100F119C101F11AC102F11BC103F1C9
:10739000000E046F000E056F0A0E066F000E076FD9
:1073A000B3EC3BF01200010104510013055101132D
:1073B000065102130751031312000101186B196BD8
:1073C0001A6B1B6B12002AC182F40401300E822753
:1073D00088EC0FF02BC182F40401300E822788EC78
:1073E0000FF02CC182F40401300E822788EC0FF0DC
:1073F0002DC182F40401300E822788EC0FF02EC1DB
:1074000082F40401300E822788EC0FF02FC182F441
:107410000401300E822788EC0FF030C182F40401A1
:10742000300E822788EC0FF031C182F40401300E57
:10743000822788EC0FF032C182F40401300E8227DB
:1074400088EC0FF033C182F40401300E822788ECFF
:107450000FF012002FC182F40401300E822788EC55
:107460000FF030C182F40401300E822788EC0FF057
:1074700031C182F40401300E822788EC0FF032C152
:1074800082F40401300E822788EC0FF033C182F4BD
:107490000401300E822788EC0FF01200060E226ED7
:1074A000060E236E060E246E222E54EF3AF0232E83
:1074B00054EF3AF0242E54EF3AF08B84020E226EF1
:1074C000020E236E020E246E222E64EF3AF0232E5B
:1074D00064EF3AF0242E64EF3AF08B941200FF0E22
:1074E000236E23C024F0030E226E8B84222E75EFB0
:1074F0003AF0030E226E242E75EF3AF08B9423C0DF
:1075000024F0030E226E222E83EF3AF0030E226E39
:10751000243E83EF3AF0232E71EF3AF0120001017E
:10752000005305E1015303E1025301E1002B52EC4A
:107530003BF097EC3CF03951006F3A51016F420E2D
:10754000046F4B0E056F000E066F000E076F93EC75
:107550003BF000C104F101C105F102C106F103C114
:1075600007F118C100F119C101F11AC102F11BC1E3
:1075700003F107B2C0EF3AF087EC3BF0C2EF3AF00C
:1075800082EC3BF000C118F101C119F102C11AF1FE
:1075900003C11BF1120097EC3CF059C100F15AC134
:1075A00001F1060E12EC0CF0E8CF04F1070E12EC1C
:1075B0000CF0E8CF05F1080E12EC0CF0E8CF06F164
:1075C000090E12EC0CF0E8CF07F182EC3BF000C1A1
:1075D00024F101C125F102C126F103C127F1290ED1
:1075E000046F000E056F000E066F000E076F93EC20
:1075F0003BF0EE0E046F430E056F000E066F000E9B
:10760000076F87EC3BF024C104F125C105F126C1C9
:1076100006F127C107F193EC3BF000C11CF101C159
:107620001DF102C11EF103C11FF1120E12EC0CF08C
:10763000E8CF04F1130E12EC0CF0E8CF05F1140EB4
:1076400012EC0CF0E8CF06F1150E12EC0CF0E8CFBE
:1076500007F10D0E006F000E016F000E026F000E9D
:10766000036F93EC3BF0180E046F000E056F000ED5
:10767000066F000E076FB3EC3BF01CC104F11DC197
:1076800005F11EC106F11FC107F187EC3BF06A0E40
:10769000046F2A0E056F000E066F000E076F82EC56
:1076A0003BF01200BF0EFA6E200E3A6F396BD89085
:1076B0000037013702370337D8B063EF3BF03A2F7A
:1076C00058EF3BF039073A070353D8B4120003319F
:1076D000070B80093F6F03390F0B010F396F80ECE7
:1076E0005FF0406F390580EC5FF0405D405F396BC3
:1076F0003F33D8B0392739333FA978EF3BF04051B9
:10770000392712000101BCEC3CF0D8B01200010195
:1077100003510719346F7FEC3CF0D89007510319DF
:1077200034AF800F12000101346BA3EC3CF0D8A001
:10773000B9EC3CF0D8B012008EEC3CF097EC3CF089
:107740001F0E366FCFEC3CF00B35D8B07FEC3CF021
:10775000D8A00335D8B01200362FA2EF3BF034B1D9
:10776000A6EC3CF012000101346B04510511061126
:1077700007110008D8A0A3EC3CF0D8A0B9EC3CF06D
:10778000D8B01200086B096B0A6B0B6BCFEC3CF0A6
:107790001F0E366FCFEC3CF007510B5DD8A4DDEF28
:1077A0003BF006510A5DD8A4DDEF3BF00551095DC1
:1077B000D8A4DDEF3BF00451085DD8A0F0EF3BF01A
:1077C0000451085F0551D8A0053D095F0651D8A0B6
:1077D000063D0A5F0751D8A0073D0B5FD890008196
:1077E000362FCAEF3BF034B1A6EC3CF0346BA3EC7F
:1077F0003CF0D890D3EC3CF007510B5DD8A40DEFD2
:107800003CF006510A5DD8A40DEF3CF00551095D2E
:10781000D8A40DEF3CF00451085DD8A01CEF3CF05B
:10782000003F1CEF3CF0013F1CEF3CF0023F1CEF1F
:107830003CF0032BD8B4120034B1A6EC3CF012009B
:107840000101346BA3EC3CF0D8B01200D8EC3CF052
:10785000200E366F003701370237033711EE33F051
:107860000A0E376FE7360A0EE75CD8B0E76EE552CE
:10787000372F32EF3CF0362F2AEF3CF034B129811C
:10788000D8901200D8EC3CF0200E366F003701374C
:107890000237033711EE33F00A0E376FE7360A0E60
:1078A000E75CD8B0E76EE552372F4EEF3CF0362F4D
:1078B00046EF3CF0D890120001010A0E346F200E02
:1078C000366F11EE29F03451376F0A0ED890E65218
:1078D000D8B0E726E732372F67EF3CF003330233A7
:1078E00001330033362F61EF3CF0E750FF0FD8A093
:1078F0000335D8B0120029B1A6EC3CF012000451B7
:1079000000270551D8B0053D01270651D8B0063DE6
:1079100002270751D8B0073D032712000051086F16
:107920000151096F02510A6F03510B6F12000101DF
:10793000006B016B026B036B12000101046B056BA2
:10794000066B076B12000335D8A012000351800BA1
:10795000001F011F021F031F003FB6EF3CF0013F55
:10796000B6EF3CF0023FB6EF3CF0032B342B03257F
:1079700012000735D8A012000751800B041F051F05
:10798000061F071F043FCCEF3CF0053FCCEF3CF057
:10799000063FCCEF3CF0072B342B072512000037B5
:1079A000013702370337083709370A370B37120018
:1079B0000101296B2A6B2B6B2C6B2D6B2E6B2F6BA4
:1079C000306B316B326B336B120001012A510F0B9C
:1079D0002A6F2B510F0B2B6F2C510F0B2C6F2D512E
:1079E0000F0B2D6F2E510F0B2E6F2F510F0B2F6F73
:1079F00030510F0B306F31510F0B316F32510F0B74
:107A0000326F33510F0B336F120000C124F101C1EB
:107A100025F102C126F103C127F104C100F105C11E
:107A200001F106C102F107C103F124C104F125C12E
:107A300005F126C106F127C107F11200000EC76E3D
:107A4000200EC66E899C9E96C69EC50EC96EFF0E00
:107A50009EB602D0E82EFCD79E96C69E000EC96E3A
:107A6000FF0E9EB602D0E82EFCD7C9CF00F69E9638
:107A7000C69E000EC96EFF0E9EB602D0E82EFCD741
:107A8000C9CF01F6898C1200000EC76E200EC66E9B
:107A9000899C9E96C69EC80EC96EFF0E9EB602D0E9
:107AA000E82EFCD79E96C69E000EC96EFF0E9EB6AF
:107AB00002D0E82EFCD7C9CF02F69E96C69E000ED5
:107AC000C96EFF0E9EB602D0E82EFCD7C9CF03F6D2
:107AD0009E96C69E000EC96EFF0E9EB602D0E82E80
:107AE000FCD7C9CF0AF69E96C69E000EC96EFF0E41
:107AF0009EB602D0E82EFCD7C9CF0BF69E96C69E46
:107B0000000EC96EFF0E9EB602D0E82EFCD7C9CF7C
:107B100012F69E96C69E000EC96EFF0E9EB602D04D
:107B2000E82EFCD7C9CF13F6898C1200000EC76E61
:107B3000200EC66E899C9E96C69EE80EC96EFF0EEC
:107B40009EB602D0E82EFCD79E96C69E000EC96E49
:107B5000FF0E9EB602D0E82EFCD7C9CF1AF69E962D
:107B6000C69E000EC96EFF0E9EB602D0E82EFCD750
:107B7000C9CF1BF69E96C69E000EC96EFF0E9EB61E
:107B800002D0E82EFCD7C9CF22F69E96C69E000EE4
:107B9000C96EFF0E9EB602D0E82EFCD7C9CF23F6E1
:107BA0009E96C69E000EC96EFF0E9EB602D0E82EAF
:107BB000FCD7C9CF2AF69E96C69E000EC96EFF0E50
:107BC0009EB602D0E82EFCD7C9CF2BF6898C1200C6
:107BD000000EC76E200EC66E899C9E96C69E240E11
:107BE000C96EFF0E9EB602D0E82EFCD79E96C69EAA
:107BF000E40EC96EFF0E9EB602D0E82EFCD7898C2B
:107C0000899C9E96C69E250EC96EFF0E9EB602D01A
:107C1000E82EFCD79E96C69E000EC96EFF0E9EB63D
:107C200002D0E82EFCD7898C899C9E96C69E200E99
:107C3000C96EFF0E9EB602D0E82EFCD79E96C69E59
:107C40005F0EC96EFF0E9EB602D0E82EFCD7898C5F
:107C5000899C9E96C69E210EC96EFF0E9EB602D0CE
:107C6000E82EFCD79E96C69EC80EC96EFF0E9EB625
:107C700002D0E82EFCD7898C899C9E96C69E260E43
:107C8000C96EFF0E9EB602D0E82EFCD79E96C69E09
:107C9000000EC96EFF0E9EB602D0E82EFCD7898C6E
:107CA00016901200000EC76E200EC66E899C9E961E
:107CB000C69E200EC96EFF0E9EB602D0E82EFCD7DF
:107CC0009E96C69E000EC96EFF0E9EB602D0E82E8E
:107CD000FCD7898C120000012650FE0AD8B479EF37
:107CE0003EF000012650FD0AD8B479EF3EF08984B9
:107CF00001D08994000EC76E220EC66E050EE82EC6
:107D0000FED7120000012650FE0AD8B490EF3EF0D4
:107D100000012650FD0AD8B490EF3EF0899401D0BE
:107D20008984050EE82EFED712006BEC3EF00001B0
:107D30002650FD0AD8B4A8EF3EF09E96C69E000ECF
:107D4000C96EFF0E9EB602D0E82EFCD7B1EF3EF012
:107D50009E96C69E010EC96EFF0E9EB602D0E82EFC
:107D6000FCD79E96C69E000EC96EFF0E9EB602D030
:107D7000E82EFCD7C9CFAFF59E96C69E000EC96E01
:107D8000FF0E9EB602D0E82EFCD7C9CFB0F59E9666
:107D9000C69E000EC96EFF0E9EB602D0E82EFCD71E
:107DA000C9CFB1F59E96C69E000EC96EFF0E9EB657
:107DB00002D0E82EFCD7C9CFB2F59E96C69E000E23
:107DC000C96EFF0E9EB602D0E82EFCD7C9CFB3F520
:107DD0009E96C69E000EC96EFF0E9EB602D0E82E7D
:107DE000FCD7C9CFB4F59E96C69E000EC96EFF0E95
:107DF0009EB602D0E82EFCD7C9CFB5F582EC3EF096
:107E000012006BEC3EF000012650FD0AD8B414EFCE
:107E10003FF09E96C69E800EC96EFF0E9EB602D0A3
:107E2000E82EFCD71DEF3FF09E96C69E810EC96ED0
:107E3000FF0E9EB602D0E82EFCD79E96C69EAFC51A
:107E4000C9FFFF0E9EB602D0E82EFCD79E96C69EB6
:107E5000B0C5C9FFFF0E9EB602D0E82EFCD79E9695
:107E6000C69EB1C5C9FFFF0E9EB602D0E82EFCD754
:107E70009E96C69EB2C5C9FFFF0E9EB602D0E82EE2
:107E8000FCD79E96C69EB3C5C9FFFF0E9EB602D014
:107E9000E82EFCD79E96C69EB4C5C9FFFF0E9EB6BF
:107EA00002D0E82EFCD79E96C69EB5C5C9FFFF0E30
:107EB0009EB602D0E82EFCD782EC3EF012006BECAE
:107EC0003EF000012650FD0AD8B472EF3FF09E96B6
:107ED000C69E070EC96EFF0E9EB602D0E82EFCD7D6
:107EE0007BEF3FF09E96C69E090EC96EFF0E9EB6B2
:107EF00002D0E82EFCD79E96C69E000EC96EFF0EDD
:107F00009EB602D0E82EFCD7C9CFAFF59E96C69E8E
:107F1000000EC96EFF0E9EB602D0E82EFCD7C9CF68
:107F2000B0F59E96C69E000EC96EFF0E9EB602D09C
:107F3000E82EFCD7C9CFB1F59E96C69E000EC96E3D
:107F4000FF0E9EB602D0E82EFCD7C9CFB2F582EC68
:107F50003EF06BEC3EF09E96C69E27C0C9FFFF0E1A
:107F60009EB602D0E82EFCD79E96C69E000EC96E25
:107F7000FF0E9EB602D0E82EFCD7C9CFB6F582EC34
:107F80003EF012006BEC3EF000012650FD0AD8B422
:107F9000D5EF3FF09E96C69E870EC96EFF0E9EB629
:107FA00002D0E82EFCD7DEEF3FF09E96C69E890EEB
:107FB000C96EFF0E9EB602D0E82EFCD79E96C69ED6
:107FC000000EC96EFF0E9EB602D0E82EFCD79E961C
:107FD000C69E800EC96EFF0E9EB602D0E82EFCD75C
:107FE0009E96C69E800EC96EFF0E9EB602D0E82EEB
:107FF000FCD79E96C69E800EC96EFF0E9EB602D01E
:10800000E82EFCD782EC3EF0120000012650FE0A5A
:10801000D8B414EF40F000012650FD0AD8B42BEF7D
:1080200040F05FEC3FF012006BEC3EF09E96C69E77
:108030008F0EC96EFF0E9EB602D0E82EFCD79E961C
:10804000C69E000EC96EFF0E9EB602D0E82EFCD76B
:1080500082EC3EF012006BEC3EF09E96C69E8E0EB9
:10806000C96EFF0E9EB602D0E82EFCD79E96C69E25
:10807000000EC96EFF0E9EB602D0E82EFCD782EC31
:108080003EF0120000012650FE0AD8B47BEF40F00B
:1080900000012650FD0AD8B4A8EF40F06BEC3EF08A
:1080A0009E96C69E28C0C9FFFF0E9EB602D0E82E3F
:1080B000FCD79E96C69E010EC96EFF0E9EB602D0DC
:1080C000E82EFCD782EC3EF06BEC3EF09E96C69E0E
:1080D000910EC96EFF0E9EB602D0E82EFCD79E967A
:1080E000C69EA50EC96EFF0E9EB602D0E82EFCD726
:1080F00082EC3EF012006BEC3EF09E96C69E28C0CD
:10810000C9FFFF0E9EB602D0E82EFCD79E96C69EF3
:10811000450EC96EFF0E9EB602D0E82EFCD782EC4B
:108120003EF06BEC3EF09E96C69E8F0EC96EFF0E23
:108130009EB602D0E82EFCD79E96C69E000EC96E53
:10814000FF0E9EB602D0E82EFCD782EC3EF0120065
:108150006BEC3EF09E96C69E28C0C9FFFF0E9EB6F1
:1081600002D0E82EFCD79E96C69E3D0EC96EFF0E2D
:108170009EB602D0E82EFCD782EC3EF06BEC3EF0CF
:108180009E96C69E8F0EC96EFF0E9EB602D0E82E3A
:10819000FCD79E96C69EA90EC96EFF0E9EB602D053
:1081A000E82EFCD782EC3EF012006BEC3EF09E967F
:1081B000C69E28C0C9FFFF0E9EB602D0E82EFCD78F
:1081C0009E96C69E810EC96EFF0E9EB602D0E82E08
:1081D000FCD782EC3EF012006BEC3EF09E96C69E01
:1081E00028C0C9FFFF0E9EB602D0E82EFCD79E968F
:1081F000C69E010EC96EFF0E9EB602D0E82EFCD7B9
:1082000082EC3EF012006BEC3EF09E96C69E910E04
:10821000C96EFF0E9EB602D0E82EFCD79E96C69E73
:10822000A50EC96EFF0E9EB602D0E82EFCD782ECDA
:108230003EF012006BEC3EF09E96C69E910EC96E0B
:10824000FF0E9EB602D0E82EFCD79E96C69E000E6C
:10825000C96EFF0E9EB602D0E82EFCD782EC3EF02F
:1082600012000501256B266B276B286B899A400E3F
:10827000C76E200EC66E9E96C69E030EC96EFF0E7A
:108280009EB602D0E82EFCD79E96C69E27C5C9FF93
:10829000FF0E9EB602D0E82EFCD79E96C69E26C53F
:1082A000C9FFFF0E9EB602D0E82EFCD79E96C69E52
:1082B00025C5C9FFFF0E9EB602D0E82EFCD79E96BC
:1082C000C69EC952FF0E9EB602D0E82EFCD7898A00
:1082D0000F01C950FF0A01E1120005012E51130AD6
:1082E00005E005012E51170A0CE012000501E00E11
:1082F000256FFF0E266F0F0E276F000E286F8AEF77
:1083000041F00501E00E256FFF0E266FFF0E276F6F
:10831000000E286F899A400EC76E200EC66E9E967C
:10832000C69E030EC96EFF0E9EB602D0E82EFCD785
:108330009E96C69E27C5C9FFFF0E9EB602D0E82EA8
:10834000FCD79E96C69E26C5C9FFFF0E9EB602D0DC
:10835000E82EFCD79E96C69E25C5C9FFFF0E9EB689
:1083600002D0E82EFCD79E96C69EC952FF0E9EB63E
:1083700002D0E82EFCD7898A0F01C950FF0A1DE000
:1083800005012E51130A05E005012E51170A0BE0D5
:1083900012000501000E256F000E266F100E276FCC
:1083A000000E286F12000501000E256F000E266FCB
:1083B000000E276F010E286F12000501256B266B3A
:1083C000276B286B05012E51130A05E005012E517C
:1083D000170A0CE012000501000E216F000E226F3B
:1083E000080E236F000E246FFFEF41F00501000E11
:1083F000216F000E226F800E236F000E246F21C5A7
:1084000000F122C501F123C502F124C503F125C500
:1084100004F126C505F127C506F128C507F1D3ECFF
:1084200039F000C125F501C126F502C127F503C1C8
:1084300028F5899A400EC76E200EC66E9E96C69E7F
:10844000030EC96EFF0E9EB602D0E82EFCD79E9694
:10845000C69E27C5C9FFFF0E9EB602D0E82EFCD7E8
:108460009E96C69E26C5C9FFFF0E9EB602D0E82E78
:10847000FCD79E96C69E25C5C9FFFF0E9EB602D0AC
:10848000E82EFCD79E96C69EC952FF0E9EB602D01D
:10849000E82EFCD7898AC950FF0A08E104C125F5F6
:1084A00005C126F506C127F507C128F5D8900501B5
:1084B00024332333223321332151E00B216F050173
:1084C00021676AEF42F022676AEF42F023676AEFA2
:1084D00042F02467FFEF41F00501200E2527E86AEE
:1084E0002623E86A2723E86A28231200E86A0501A0
:1084F0002E51130A06E005012E51170A0BE0020E59
:10850000120005012851000A03E12751F00B07E092
:10851000010E120005012851000A01E0010E1200AF
:1085200029C500F12AC501F12BC502F12CC503F1C3
:1085300025C504F126C505F127C506F128C507F1B3
:1085400082EC3BF003BF120076EC42F0D8A408EFB7
:1085500043F0899A400EC76E200EC66E9E96C69E48
:10856000060EC96EFF0E9EB602D0E82EFCD7898A91
:10857000899A9E96C69E020EC96EFF0E9EB602D0C6
:10858000E82EFCD79E96C69E27C5C9FFFF0E9EB655
:1085900002D0E82EFCD79E96C69E26C5C9FFFF0EC8
:1085A0009EB602D0E82EFCD79E96C69E25C5C9FF72
:1085B000FF0E9EB602D0E82EFCD79E96C69E000EF9
:1085C000C96EFF0E9EB602D0E82EFCD7898A899A22
:1085D0009E96C69E050EC96EFF0E9EB602D0E82E70
:1085E000FCD79E96C69EC952FF0E9EB602D0E82EBC
:1085F000FCD7C9B0F1EF42F0898A0501200E25278A
:10860000E86A2623E86A2723E86A282390EF42F0E5
:108610001200899A400EC76E200EC66E9E96C69EA8
:10862000060EC96EFF0E9EB602D0E82EFCD7898AD0
:10863000899A9E96C69EC70EC96EFF0E9EB602D040
:10864000E82EFCD7898A0501256B266B276B286BE2
:108650001200899A400EC76E200EC66E9E96C69E68
:10866000050EC96EFF0E9EB602D0E82EFCD79E9670
:10867000C69EC952FF0E9EB602D0E82EFCD7C9CFC7
:1086800037F5898A1200899A400EC76E200EC66E91
:108690009E96C69EB90EC96EFF0E9EB602D0E82EFB
:1086A000FCD7898A1200899A400EC76E200EC66ECA
:1086B0009E96C69EAB0EC96EFF0E9EB602D0E82EE9
:1086C000FCD7898AFF0EE82EFED7120076EC42F026
:1086D000D8A41200899A400EC76E200EC66E9E96D0
:1086E000C69E030EC96EFF0E9EB602D0E82EFCD7C2
:1086F0009E96C69E27C5C9FFFF0E9EB602D0E82EE5
:10870000FCD79E96C69E26C5C9FFFF0E9EB602D018
:10871000E82EFCD79E96C69E25C5C9FFFF0E9EB6C5
:1087200002D0E82EFCD79E96C69EC952FF0E9EB67A
:1087300002D0E82EFCD7898A0F01C950FF0AD8A4BD
:10874000E1EF46F00501FE0E376F0501FF0E536F96
:10875000FF0E546FFF0E556FFF0E566F15A637991B
:10876000158695EC3EF0AFC538F5B0C539F5B1C505
:108770003AF5B2C53BF5B3C53CF5B4C53DF5B5C555
:108780003EF50784BAC166F1BBC167F1BCC168F1AF
:10879000BDC169F14BC14FF14CC150F14DC151F117
:1087A0004EC152F157C159F158C15AF10001175049
:1087B000010AD8B4EAEF43F000011750020AD8B416
:1087C0000FEF44F000011750040AD8B434EF44F01E
:1087D000E1EF46F00501476B486B496B4A6B0501B9
:1087E0004B6B4C6B4D6B4E6B05014F6B506B516B74
:1087F000526B8BA0379B58EC2CF000C1DAF101C111
:10880000DBF102C1DCF103C1DDF100C13FF501C1C3
:1088100040F502C141F503C142F553EF44F00501B3
:10882000476B486B496B4A6B05014B6B4C6B4D6B4F
:108830004E6B05014F6B506B516B526B58EC2CF02B
:1088400000C1DAF101C1DBF102C1DCF103C1DDF1EC
:1088500055EC2DF000C147F501C148F502C149F5BD
:1088600003C14AF5E1EF46F0379BDAC13FF5DBC1C2
:1088700040F5DCC141F5DDC142F558EC2CF000C1FA
:108880004BF501C14CF502C14DF503C14EF555EC58
:108890002DF000C14FF501C150F502C151F503C1E2
:1088A00052F553EF44F0050161675EEF44F06267F3
:1088B0005EEF44F063675EEF44F0646762EF44F09C
:1088C00077EF44F0DAC100F1DBC101F1DCC102F164
:1088D000DDC103F161C504F162C505F163C506F1AF
:1088E00064C507F182EC3BF003BFE1EF46F059C1EC
:1088F00043F55AC144F5B9C545F5DAEC38F036C64A
:1089000049F537C64AF5060140678EEF44F04167E6
:108910008EEF44F042678EEF44F0436792EF44F0ED
:10892000A3EF44F097EC3CF09DEC3CF036C600F130
:1089300037C601F140C604F141C605F182EC3BF0B7
:1089400003AFE1EF46F00101036B026B1AC600F1C1
:108950001BC601F101AFB1EF44F0FF0E026FFF0E35
:10896000036F0101076B066B1CC604F11DC605F100
:1089700005AFBFEF44F0FF0E066FFF0E076F87ECE9
:108980003BF00101076B066B1EC604F11FC605F123
:1089900005AFCFEF44F0FF0E066FFF0E076F87ECB9
:1089A0003BF00101076B066B20C604F121C605F1FF
:1089B00005AFDFEF44F0FF0E066FFF0E076F87EC89
:1089C0003BF0D89001010333023301330033D890D8
:1089D0000101033302330133003300C14BF501C100
:1089E0004CF50101036B026B22C600F123C601F1B5
:1089F00001AFFFEF44F0FF0E026FFF0E036F0101A6
:108A0000076B066B24C604F125C605F105AF0DEF13
:108A100045F0FF0E066FFF0E076F87EC3BF001017C
:108A2000076B066B26C604F127C605F105AF1DEFDF
:108A300045F0FF0E066FFF0E076F87EC3BF001015C
:108A4000076B066B28C604F129C605F105AF2DEFAB
:108A500045F0FF0E066FFF0E076F87EC3BF0D890D6
:108A600001010333023301330033D8900101033392
:108A700002330133003300C14DF501C14EF5010150
:108A8000036B026B2AC600F12BC601F101AF4DEF5B
:108A900045F0FF0E026FFF0E036F0101076B066BBF
:108AA0002CC604F12DC605F105AF5BEF45F0FF0EB6
:108AB000066FFF0E076F87EC3BF00101076B066B3B
:108AC0002EC604F12FC605F105AF6BEF45F0FF0E82
:108AD000066FFF0E076F87EC3BF00101076B066B1B
:108AE00030C604F131C605F105AF7BEF45F0FF0E4E
:108AF000066FFF0E076F87EC3BF0D8900101033340
:108B0000023301330033D8900101033302330133C0
:108B1000003300C14FF501C150F50101036B026B39
:108B200002C600F103C601F101AF9BEF45F0FF0E55
:108B3000026FFF0E036F0101076B066B04C604F1A1
:108B400005C605F105AFA9EF45F0FF0E066FFF0E54
:108B5000076F87EC3BF00101076B066B06C604F15B
:108B600007C605F105AFB9EF45F0FF0E066FFF0E22
:108B7000076F87EC3BF00101076B066B08C604F139
:108B800009C605F105AFC9EF45F0FF0E066FFF0EF0
:108B9000076F87EC3BF0D8900101033302330133B8
:108BA0000033D8900101033302330133003300C195
:108BB00051F501C152F50101036B026B0AC600F1C8
:108BC0000BC601F101AFE9EF45F0FF0E026FFF0E9A
:108BD000036F0101076B066B0CC604F10DC605F1AE
:108BE00005AFF7EF45F0FF0E066FFF0E076F87EC3E
:108BF0003BF00101076B066B0EC604F10FC605F1D1
:108C000005AF07EF46F0FF0E066FFF0E076F87EC0C
:108C10003BF00101076B066B10C604F111C605F1AC
:108C200005AF17EF46F0FF0E066FFF0E076F87ECDC
:108C30003BF0D89001010333023301330033D89065
:108C40000101033302330133003300C153F501C185
:108C500054F50101036B026B12C600F113C601F15A
:108C600001AF37EF46F0FF0E026FFF0E036F0101F9
:108C7000076B066B14C604F115C605F105AF45EF89
:108C800046F0FF0E066FFF0E076F87EC3BF0010109
:108C9000076B066B16C604F117C605F105AF55EF55
:108CA00046F0FF0E066FFF0E076F87EC3BF00101E9
:108CB000076B066B18C604F119C605F105AF65EF21
:108CC00046F0FF0E066FFF0E076F87EC3BF0D89063
:108CD00001010333023301330033D8900101033320
:108CE00002330133003300C155F501C156F50501CA
:108CF000210E326F899A400EC76E200EC66E9E9668
:108D0000C69E060EC96EFF0E9EB602D0E82EFCD798
:108D1000898A899A9E96C69E020EC96EFF0E9EB6DD
:108D200002D0E82EFCD79E96C69E27C5C9FFFF0E2F
:108D30009EB602D0E82EFCD79E96C69E26C5C9FFD9
:108D4000FF0E9EB602D0E82EFCD79E96C69E25C585
:108D5000C9FFFF0E9EB602D0E82EFCD725EE37F0F5
:108D6000322F02D0BFEF46F09E96C69EDECFC9FFDF
:108D7000FF0E9EB602D0E82EFCD7B0EF46F0898AEF
:108D8000899A9E96C69E050EC96EFF0E9EB602D0AB
:108D9000E82EFCD79E96C69EC952FF0E9EB602D004
:108DA000E82EFCD7C9B0CAEF46F0898A0501200E2B
:108DB0002527E86A2623E86A2723E86A28234EEC59
:108DC0003AF015900794120021C500F122C501F177
:108DD00023C502F124C503F1899A400EC76E200E07
:108DE000C66E9E96C69E0B0EC96EFF0E9EB602D034
:108DF000E82EFCD79E96C69E02C1C9FFFF0E9EB606
:108E000002D0E82EFCD79E96C69E01C1C9FFFF0E78
:108E10009EB602D0E82EFCD79E96C69E00C1C9FF22
:108E2000FF0E9EB602D0E82EFCD79E96C69EC95273
:108E3000FF0E9EB602D0E82EFCD725EE37F00501D6
:108E4000200E326F9E96C69EC952FF0E9EB602D06D
:108E5000E82EFCD7C9CFDEFF322F22EF47F0898AF8
:108E60001200899A400EC76E200EC66E9E96C69E50
:108E7000900EC96EFF0E9EB602D0E82EFCD79E96CD
:108E8000C69E000EC96EFF0E9EB602D0E82EFCD71D
:108E90009E96C69E000EC96EFF0E9EB602D0E82EAC
:108EA000FCD79E96C69E000EC96EFF0E9EB602D0DF
:108EB000E82EFCD79E96C69EC952FF0E9EB602D0E3
:108EC000E82EFCD7C9CF2DF59E96C69EC952FF0E3F
:108ED0009EB602D0E82EFCD7C9CF2EF5898A1200A3
:108EE00095EC3EF005012F51010A61E005012F517B
:108EF000020A16E005012F51030A1BE005012F515C
:108F0000040A26E005012F51050A2DE005012F5125
:108F1000060A3BE005012F51070A41E0D7EF47F071
:108F200015B01200602FD5EF47F05FC560F5D7EFA1
:108F300047F0B0C500F101010F0E0017010100510B
:108F4000000A35E001010051050A31E0D5EF47F094
:108F5000B0C500F101010F0E001701010051000A18
:108F600026E0D5EF47F00501B051000A20E00501E9
:108F7000B051150A1CE00501B051300A18E0050196
:108F8000B051450A14E0D5EF47F00501B051000A91
:108F90000EE00501B051300A0AE0D5EF47F00501B7
:108FA000B051000A04E0D5EF47F01590120015808B
:108FB00012008B904EEC3AF0B9C5E8FFD70802E3F7
:108FC0004EEC3AF0B9C5E8FFC80802E34EEC3AF0BF
:108FD000B9C5E8FFB90802E34EEC3AF0B9C5E8FFBD
:108FE000AA0802E34EEC3AF0B9C5E8FF9B0802E399
:108FF0004EEC3AF043EC43F0F29CF29E8B94C69A0E
:10900000C29052EC3EF09482948C720ED36ED3A434
:10901000FED789968A909390F29AF2949D909E90B2
:109020009D929E92F298F29205EC40F0FF0EE8CFEE
:1090300000F0E82EFED7002EFCD7F290F286815089
:10904000FF0EE82EFED7F29081A829EF48F0F29E9D
:109050000300700ED36EF296F290158403806FECCD
:069060003AF048EF0CF0AD
:10BF0000E844F926000C160C2B0C3F0C520C640C68
:10BF1000760C860C960CA50CB30CC10CCF0CDC0C6B
:06BF2000E80CF40C000C1B
:0200000400F00A
:0100C800FE39
:00000001FF
